:020000040000fa
:080000009a0704000000000053
:020000040000fa
:020000040002f8
:04afe000dfff00008f
:020000040000fa
:020000040002f8
:04afe400ffff00006b
:020000040000fa
:020000040002f8
:04afe80078ff0000ee
:020000040000fa
:020000040002f8
:04afec007dff0000e5
:020000040000fa
:020000040002f8
:04aff00078ff0000e6
:020000040000fa
:1000080000000000000000000000000000000000e8
:10001800920700000000000000000000000000003f
:10002800c20b00000000000000000000f60b0000fa
:100038000000000000000000000000003c0c000070
:10004800680c00000000000000000000620d0000c5
:100058000000000000000000000000000000000098
:100068000000000000000000000000000000000088
:100078000000000000000000000000000000000078
:10008800000000000000000000000000980c0000c4
:100098000000000000000000000000000000000058
:1000a8000000000000000000000000000000000048
:1000b8000000000000000000000000000000000038
:1000c8000000000000000000000000000000000028
:1000d8000000000000000000000000000000000018
:1000e8000000000000000000000000000000000008
:1000f80000000000000000000000000000000000f8
:1001080000000000000000000000000000000000e7
:1001180000000000000000000000000000000000d7
:10012800000000009a0d0000000000000000000020
:1001380000000000000000000000000000000000b7
:1001480000000000000000000000000000000000a7
:100158000000000000000000000000000000000097
:100168000000000000000000000000000000000087
:100178000000000000000000000000000000000077
:100188000000000000000000000000000000000067
:100198000000000000000000ce0d0000fa0d000075
:1001a800260e000000000000000000000000000013
:1001b8000000000000000000000000000000000037
:1001c8000000000000000000000000000000000027
:1001d8000000000000000000000000000000000017
:1001e8000000000000000000000000000000000007
:1001f80000000000000000000000000000000000f7
:1002080000000000000000000000000000000000e6
:1002180000000000000000000000000000000000d6
:1002280000000000000000000000000000000000c6
:1002380000000000000000000000000000000000b6
:1002480000000000000000000000000000000000a6
:100258000000000000000000000000000000000096
:100268000000000000000000000000000000000086
:0c0278000000000000000000000000007a
:020000040000fa
:10040000fdd1bf00fc51b7004220af00fc71ec00f1
:10041000fdd1d600fdd1b60000c0d200fdd1bf0095
:1004200000c0fd00fdf1b700fcd1bf0000c0fd0021
:100430000040d200fdd1b600fdd1bf0000c0fd00dc
:10044000fdf1b7001040b200fcf1d600fcf1b6009f
:10045000fdf1d600e08f800000000600803e200005
:10046000030007008100e900fcff3a0000000600dd
:10047000831f7800c20320000400bc006601510005
:10048000e0815900f23fb1000380b1000600350061
:10049000ee03090000000000423fb1000380b100fc
:1004a000fbff3d001200b000223fb000020035000b
:1004b0000280090000000000cf0178000000060063
:1004c000839f68000100e00002003d006000100012
:1004d000e08018000300e00002003d006001110010
:1004e000e0811900050007004f00e00002003b001a
:1004f00060001000e080180000000600861f7800f1
:100500006022b800060220000000d0008180d200e6
:100510000482d2008582d2000000a00002025200b4
:1005200083825a00030031000202420083824a00a3
:100530000000a1000603e900f3ff3a004f03780032
:10054000000006000001eb00869fbe00889fbe00f1
:100550008a9fbe008c9fbe00820578000004be000a
:10056000240207000800be006420e10007003900f3
:1005700002003a00f1ff2f00f0ff27000160a00009
:100580001202200012908800560037006120e1001e
:1005900003003a000b00a70001f8230051003700c8
:1005a00001f0a10002002100936424005200070022
:1005b0000800be0005003500b2fd2000930c2400a9
:1005c00004002000690007000004be000005eb00e5
:1005d0000b00a6004f0dde0001f0a1000004be00dc
:1005e00032982f0023ea2300520107000001eb009c
:1005f000030020000b00a70003f82300ac00070055
:10060000810107000000a7000a00a200c401070042
:100610000b00e000030032000200200003f0230082
:10062000a200070001f0a2000006be0002002000a8
:10063000930424003f0107000801be009c0007004e
:10064000809fbe000c00be0022a22a00d3a7230078
:10065000380107004f01be00950007000004be00ee
:1006600001f0a100020020000398230022000700ef
:100670000800be00190035000001be002d01070072
:100680000006be00b2c52900e3622300290107006d
:1006900022222b00f3942b00850007000c01be00e2
:1006a00024010700e273280083c0230080000700b4
:1006b0000c01be001f01070042aa2a00a3e22b0082
:1006c0007b0007000c01be001a0107000801be00f4
:1006d000180107000801be00750007000a00a70006
:1006e00001f0a2004f06be004f05be004f04be0041
:1006f0004f03be000000060014002000889fbe00cb
:100700008a9fbe00841f7800b20107004f00780066
:1007100011003300f0ff2f00838f6c0006003b00b8
:10072000040565000a00a7000800370009f0a600cc
:100730001000200008003700820f5400838f5c00f7
:10074000030039001000200001003e0000002000de
:1007500009f0a7000000ea004f05be004f04be00ec
:100760000000e0000000060014002000869fbe008c
:10077000889fbe008a9fbe008c9fbe004f26dd0072
:1007800094010700d60133006120e10043003200ec
:100790006250e10041003e003e0039006420e1006b
:1007a0003c003200058255000f003b000402e800c7
:1007b00038003a00800f5300818f5b003500340011
:1007c0000800be0003f0a10001f0a60003f0a000a5
:1007d0000cf0a70036000700ca01370006034300eb
:1007e00087834b000c4646000005530081855b0063
:1007f000020033000a03be000c00a0000402e9005e
:10080000f6ff3b00850578000602430087824b0017
:1008100004003a006000b80009f0a70001f0a00051
:10082000b80137000002520081825a000704e0003c
:10083000040033000603430087834b008b05e90067
:10084000faff3700090578000604be000203be0067
:100850006011b8007c010700e00f5200e08f5a00e1
:100860000700350002003c000c08a3000400320021
:100870000601be0003f0a0000cf0a7000c0007006a
:100880000a85680001f0a1000af0a70001f0a000ad
:100890009c0137000800be009a01370010022000ba
:1008a0000cf0a600109088009b01370003f0a20016
:1008b000869fbe00889fbe008a9fbe008c9fbe00a0
:1008c00044010700860133006450e1004f0032000c
:1008d0006420e1005200320003826c0007003b00fc
:1008e0000905d0000306d000820f54000c065d00fd
:1008f0000200390002003200890178000306780006
:100900008582550004003d000003fd008103fd00c9
:100910008502ea008b854200840f720002003b00d2
:1009200060001000e08018006011b8000005eb00c6
:100930007a28e1000a00390006007800c75ddd0072
:10094000f707b200878075002d00370082817100a3
:100950000a017800610560008180d1000080d30029
:100960008502e900f9ff3b00060440008784480047
:1009700002003b0060041400e0841c000988a3000e
:10098000070032008a817100828171006101640078
:100990008904d1000884d3008b05e80017003700d4
:1009a0000978a30013003a000b00e00013003400a4
:1009b0008b05e9000804440089844c000a44740053
:1009c0000978a3000d003a000b00e0000700340096
:1009d0008b05e9000804440089844c0001003a00ba
:1009e0000b0020000978a300f7ff32000001eb00a4
:1009f00002003700828171000a01780012010700ad
:100a00000cf0a70001f0a0003e0137006420e100d7
:100a100002003a00838f6c003f0133000801be00e2
:100a20000200be0037013700869fbe00889fbe00cf
:100a30008a9fbe008c9fbe00e6000700280133009d
:100a400003866c006450e1002e0032006420e10057
:100a5000330032006150e1002f0032006120e100dc
:100a60003100320085855500eb07b00009002000f9
:100a700008042000050037000804440089844c0065
:100a80000a0031000603430087834b000001530036
:100a900081815b00f8ff33000203be000800a00064
:100aa0000804440089844c00f6ff3900c639dd0093
:100ab0008301730001003200130020008904d1007b
:100ac0000884d3000998a300050032000800a7009d
:100ad0000300a0008904d1000884d3008b05e8003e
:100ae0008904d1000884d3000001eb000281d20008
:100af000d500070001f0a1000cf0a70001f0a00054
:100b0000000137006420e100030132000801be004b
:100b10000200be00f7ff37006120e100fe00320056
:100b20006000b800f3ff37000000200001f8270044
:100b3000f0ff3700869fbe00889fbe008a9fbe00e0
:100b40008c9fbe00a3000700e500330003866c0005
:100b50006450e100240032006420e10027003200ec
:100b60006150e100220032006120e10021003200ea
:100b70008b854200eb07b1000134b800003ab800a1
:100b80000804420089844a00013ab8000030b800e5
:100b90008880400009014a00040033000000400042
:100ba00081804800020149008b05e900c909dd0088
:100bb000830170000100320013002000c814de0021
:100bc0004814dd004709de001200b200c808de004c
:100bd000088470009c00070001f0a1000cf0a70041
:100be00001f0a000c70037006120e100ca00320018
:100bf0000801be000200be00f7ff37006150e100af
:100c0000fcff3a00c4003700829fbe000001be0016
:100c1000780007000470a70003f0a1006509b10087
:100c2000180032000e0035006828e100070035008a
:100c3000f0ff2f00f1ff27000300e00015003b004c
:100c4000010028004f01be00000005000000400028
:100c5000818048008502e900fcff3a000900370066
:100c6000f88f420003003c008000eb004f01be0003
:100c7000000005008100d1000080d3008502e8005b
:100c8000fcff3a000300e00002003b00600010009f
:100c9000e08018004f01be0000000600829fbe00e9
:100ca0000001be00530007000470a70003f0a1007c
:100cb00003f8a30015003a006509b10011003200e5
:100cc0000a0035006928e100030035000100280012
:100cd0004f01be0000000500000040008180480078
:100ce0008502e900fcff3a0006003700f88f420059
:100cf000060035008100d1000080d3008502e800a5
:100d0000fcff3a004f01be00000006008000eb002f
:100d10004f01be00000005000080fb008000eb00da
:100d2000829fbe00889fbe008a9fbe00010578009a
:100d30000100e0000400350008003c000000e00075
:100d4000200032000500370060001000e08018002d
:100d500002003b0001f024001a0037000004be002e
:100d60006011b8006b0920000982cf000200390031
:100d70000882cf000441b000694252000e003200e8
:100d800008003b0082817100610164008904d10088
:100d90000884d3008b05e8000442e800f9ff3a001c
:100da000050037000804440089844c008b05e900e5
:100db0000442e900fbff3a00230007000af0a70005
:100dc00001f0a0004f05be004f04be004f01be0061
:100dd000000006000004be00060007000003be007d
:100de0000405be000200be0002000700844f75002b
:100df00000000600c70ade00f107b200f50fb200de
:100e000008003200e1cf4200020032000170a00071
:100e100024000500810f7000010032000408050065
:100e200044000500810f700002003a001400050024
:100e30008502e9000000400081c04800fcff3b0043
:100e40000170a00024000500810020006180550091
:100e50000b003d000b00200061fe2f000100e100af
:100e60001d00340082817100610164008904d10099
:100e70000884d3000000e800faff3a007100200067
:100e8000610064000300700002006000090032008d
:100e900061044400e0844c000988a500050032008c
:100ea0008b05e8006808e10002003a008904d100df
:100eb0000884d300f20f20000258e10005003d0035
:100ec000c75ddd00f907b200898075000800780071
:100ed000000006000bf827008b00780000000500da
:100ee0000200be006450e100050036006420e1000d
:100ef000020036000968a30001003a000800be00a5
:100f00000160a0004f06be004f05be004f04be00aa
:100f10004f03be0000000600f0ff2f00f1ff270086
:100f2000f8ff37000020ef000220ef00c088a90082
:100f3000004006000f002100202b21000001880046
:100f4000000000000000eb00000778000c00090022
:100f5000002f78000007eb005420ef000e2eef006a
:100f60001e2eef000000eb00411f21000b1e0900a8
:100f70008018780040a7a900a100200037fd0700d5
:100f8000e0022000303a880044e7a90044c7a900e5
:100f90004407a9004427a9004447a9004467a900c1
:100fa0004487a900300020000600fc0031742000b6
:100fb00082072000a3092000824878008348780037
:100fc00080487800113a8000618070000600fc00c3
:100fd00021742000620420007305200082487800fc
:100fe00083487800804878004427ef00e002200022
:100ff000303a8800300020000d00fc0031742000e1
:1010000082072000a30920008248780083487800e6
:101010008048780000002000217420006204200035
:101020007305200082487800834878008048780063
:1010300042a7ae00feff3700813e200007fd0700fb
:1010400010c0b30086e6b70090c2b300c4e6b70094
:101050000002200000708800007825008070880061
:1010600010aea90010cea9004008a9004028a90090
:101070004048a8002008a8000008a900c208a8004d
:1010800080c0b300c8e8b7004188a90041a8a80003
:1010900041c8a800001020001008880004a1a90081
:1010a0000481a90005e1a8000068a90011a1a90018
:1010b0001061a9001021a90010a1a8001081a800aa
:1010c0000621ef00008020006008880000e8a900e9
:1010d0004388a80043a8a90043c8a90020e8a900a4
:1010e00011e1a90013a1a90013e1a8001221a90090
:1010f00012a1a8001281a8004408a8004428a90051
:101100004448a9000a21ef000ea1ef000108a90040
:101110002108a80013e1a8001fe1a8001fa1a90051
:101120001ec1a9001ea1a8001e81a9001e61a90060
:101130001e21a9001421ef0050412100d008880091
:101140004d88a8004da8a8004dc8a9000368a900b3
:101150002368a8004e08a9004e28a9004e48a900ff
:101160000388a9002388a9002002a9002022a90041
:101170002042a90020a2a9002062a9002082a90083
:1011800020e2a9002102a9002122a9007007200065
:101190004011880022a2a90022c2a90022e2a900cf
:1011a00021e2a8002182a9004588a80045a8a9003d
:1011b00045c8a8002168a8002828a8002bc8a900b5
:1011c0002be8a9002c08a9000bc8a9000be8a9006e
:1011d0000c08a90001eca90001aca900016ca90050
:1011e000014ca800012ca900010ca90000eca900e9
:1011f000008ca90000aca90000cca900000ca9003b
:10120000002ca900004ca900006ca900202cef00c4
:10121000402cef00602cef0020eca800200ca80070
:1012200040eca800400ca80060eca800600ca800ee
:10123000f07f200020608800020ca900022ca90089
:10124000024ca9000040200030618800462cef00cd
:10125000662cef00282cef00482cef00682cef00e4
:101260000aacef0023eca80023cca80043eca800b4
:1012700043cca90063eca80063cca90023aca9006f
:10128000238ca900dabc2a001b32240030002c0079
:10129000fa608800fb60880020618800dabc2a00c0
:1012a0001b32240020002c00fa608800fb608800bc
:1012b00010618800dabc2a001b32240030002c00a8
:1012c000fa608800fb60880020628800dabc2a008f
:1012d0001b32240000002800fa608800fb608800b0
:1012e00010628800dabc2a001b32240030002c0077
:1012f000fa608800fb60880020638800dabc2a005e
:101300001b32240000002800fa608800fb6088007f
:1013100010638800a70037003f003700002020003e
:10132000006188000020200000628800002020006a
:1013300000638800020ca900022ca800024ca8003f
:1013400004acef0028acef0048acef0068acef0055
:10135000262cef00462cef00662cef000aacef00c5
:1013600023eca80023cca90043eca80043cca9009f
:1013700063eca80063cca900dabc2a001b3224006d
:1013800030002c00fa608800fb6088002061880033
:10139000dabc2a001b32240000002800fa60880012
:1013a000fb60880010618800dabc2a001b32240030
:1013b00030002c00fa608800fb6088002062880002
:1013c000dabc2a001b32240000002800fa608800e2
:1013d000fb60880010628800dabc2a001b322400ff
:1013e00030002c00fa608800fb60880020638800d1
:1013f000dabc2a001b32240000002800fa608800b2
:10140000fb6088001063880011eea90011aea900ee
:10141000116ea9006700370035003700001020006a
:101420000061880000102000006288000010200089
:1014300000638800020ca900022ca800024ca8003e
:101440000a2cef0004acef00282cef0050552500cb
:1014500040628800a0aa2a0040638800dabc2a0003
:101460001b32240030002c00fa608800fb608800ea
:1014700020618800dabc2a001b32240000002c0006
:10148000fa608800fb60880010618800dabc2a00de
:101490001b32240030002c00fa608800fb608800ba
:1014a00020628800dabc2a001b32240000002c00d5
:1014b000fa608800fb60880010628800dabc2a00ad
:1014c0001b32240030002c00fa608800fb6088008a
:1014d00020638800dabc2a001b32240000002c00a4
:1014e000fa608800fb6088001063880031003700d4
:1014f000300037000010200000618800001020003c
:1015000000628800020ca900022ca800024ca8006e
:101510000a2cef0004acef00282cef0000002400a0
:1015200040628800dabc2a001b32240030002c0004
:10153000fa608800fb60880020618800dabc2a001d
:101540001b32240000002c00fa608800fb60880039
:1015500010618800dabc2a001b32240030002c0005
:10156000fa608800fb60880020628800dabc2a00ec
:101570001b32240000002c00fa608800fb60880009
:1015800010628800dabc2a001b32240030002c00d4
:10159000fa608800fb60880020638800dabc2a00bb
:1015a0001b32240000002c00fa608800fb608800d9
:1015b00010638800218ca900418ca900618ca900ce
:1015c000216ca900416ca900616ca900214ca90003
:1015d000414ca900614ca90020eca80040eca800f7
:1015e00060eca8003e2cef005e2cef007e2cef009c
:1015f00001eca800e0482100f0908800c08821009c
:1016000000918800e088210010918800c0c8210066
:1016100020918800e0c8210030918800c008220095
:1016200040918800e008220050918800c0482200c4
:1016300060918800e048220070918800c0882200f4
:1016400080918800e088220090918800c0c8220024
:10165000a0918800e0c82200b0918800c008230053
:10166000c0918800e0482100d0918800c088210006
:10167000e0918800e0482200f0918800c0882200b4
:1016800000928800e048220010928800c088220062
:1016900020928800e048220030928800c088220012
:1016a00040928800d091800070908800e091800086
:1016b0008090880010928000b09088002092800076
:1016c000c0908800f0918000909088000092800087
:1016d000a090880030928000d090880040928000d6
:1016e000e0908800e0182300d0928800e0282300d2
:1016f000e0928800e0382300f0928800e048230060
:1017000000938800e058230010938800e0682300cd
:1017100020938800e0782300309388000000eb00dd
:10172000e1882300ff000900805878007572ef00ff
:101730007672ef000432ef0085f2ef00d42a070042
:1017400026060700250a0700240e07006b12070073
:101750006b1807006b1e070090240700ec3821006f
:10176000e01823007f000900301e7800b12a07002e
:10177000ea05070047350700e8040700b904070039
:1017800054013700ff3ffc004200f8003600f8002b
:101790004400f8008e1f78000e0020000d000900a4
:1017a000be1f78003200f8000100fc000008a9000c
:1017b0002068a9000068a90000402000306188006e
:1017c000ff3ffc003200f900ae0120000d000900cf
:1017d0004f1778004f0778004400f9003600f900f1
:1017e0004200f9000100fc0000400600ff3ffc0041
:1017f0004200f8003600f8004400f8008e1f780020
:101800000e0020000d000900be1f78003200f80015
:101810000100fc000068a900a09280004a12b400f8
:101820001008880062908000120078003061880003
:101830000cb2ec005090800061908000808f5000ce
:10184000020036004090800060908800ff3ffc005e
:101850003200f900ae0120000d0009004f1778009a
:101860004f0778004400f9003600f9004200f90003
:101870000100fc0000400600ff3ffc004200f800b1
:101880003600f8004400f8008e1f78000e0020009b
:101890000d000900be1f78003200f8000100fc00b6
:1018a00000e8a900ff3ffc003200f900ae01200073
:1018b0000d0009004f1778004f0778004400f90029
:1018c0003600f9004200f9000100fc00004006006b
:1018d000ff3ffc004200f8003600f8004400f8002a
:1018e0008e1f78000e0020000d000900be1f78003a
:1018f0003200f8000100fc000108a900128eaa00c5
:10190000108ea900ff3ffc003200f900ae0120005c
:101910000d0009004f1778004f0778004400f900c8
:101920003600f9004200f9000100fc00004006000a
:10193000ff3ffc004200f8003600f8004400f800c9
:101940008e1f78000e0020000d000900be1f7800d9
:101950003200f800f411f800f611f800f811f80060
:10196000fa11f8000100fc000368a9008812ae001b
:101970002d0037008b72ec00f0c1b3008b72b60003
:1019800087d2bf000080fb0000004000e108230078
:1019900060807800a08f88008bd2bf000080fb00a1
:1019a000e198230060c07800f6f1b700a08f8000b6
:1019b000cf80de000001be00f6d1bf000000fb00ba
:1019c000cf80de00020ab800800278000200b80072
:1019d00081004200032ab800810042000001be00dd
:1019e00089d2bf000000fb00cf80de00020ab800f1
:1019f000800278000200b80081004200032ab8008b
:101a000081004200809388009193880002002100a9
:101a1000030020008093800091938000a8fa0700c3
:101a200060928800060037008b72ef004c12e200d3
:101a3000010034004c32ed004df2af004c32ec00ae
:101a400087d2bf000080fb0000004000e138210089
:101a500060807800a08f880060928000f411b4004c
:101a6000c08f880020908000f811b4005092880048
:101a70008ad2bf000080fb0000004000e128210066
:101a800060807800d0088800ff3ffc00fa11f90060
:101a9000f811f900f611f900f411f9003200f9001b
:101aa000ae0120000d0009004f1778004f077800a5
:101ab0004400f9003600f9004200f9000100fc0082
:101ac00000400600ff3ffc004200f8003600f8002e
:101ad0004400f8008e1f78000e0020000d00090061
:101ae000be1f78003200f8000100fc000168a90068
:101af0007572ec0075d2bf008080fb003011800051
:101b0000e288230080707900ff3ffc003200f9007a
:101b1000ae0120000d0009004f1778004f07780034
:101b20004400f9003600f9004200f9000100fc0011
:101b300000400600ff3ffc004200f8003600f800bd
:101b40004400f8008e1f78000e0020000d000900f0
:101b5000be1f78003200f8000100fc000828a90030
:101b60002242ae00000037002222af002222a9004c
:101b7000ff3ffc003200f900ae0120000d0009001b
:101b80004f1778004f0778004400f9003600f9003d
:101b90004200f9000100fc0000400600ff3ffc008d
:101ba0004200f8003600f8004400f8008e1f78006c
:101bb0000e0020000d000900be1f78003200f80062
:101bc0000100fc000bc8a900ff3ffc003200f90037
:101bd000ae0120000d0009004f1778004f07780074
:101be0004400f9003600f9004200f9000100fc0051
:101bf00000400600ff3ffc004200f8003600f800fd
:101c00004400f8008e1f78000e0020000d0009002f
:101c1000be1f78003200f8000100fc000be8a900ac
:101c2000ff3ffc003200f900ae0120000d0009006a
:101c30004f1778004f0778004400f9003600f9008c
:101c40004200f9000100fc0000400600ff3ffc00dc
:101c50004200f8003600f8004400f8008e1f7800bb
:101c60000e0020000d000900be1f78003200f800b1
:101c70000100fc000c08a900ff3ffc003200f90045
:101c8000ae0120000d0009004f1778004f077800c3
:101c90004400f9003600f9004200f9000100fc00a0
:101ca0000040060076d2bf007552e3000700320004
:101cb0007672ec0076d2bf000080fb00e188230042
:101cc00060c0780077f2b7000100370077f2ef00cc
:101cd00000000600f3ff070040ceb3007752b500c6
:101ce00006003900e0cfb3007752b500010039009b
:101cf000010037007872ef004101370077f2ae0043
:101d0000370037007872ef0030c8b3007752e30035
:101d100005003a0077d2bf0078f2b70079f2ef0001
:101d20007af2ef002d00370030c9b3007752e3009c
:101d300005003a0077d2bf0078f2b7007bf2ef00df
:101d40007cf2ef002500370030cab3007752e30081
:101d500005003a0077d2bf0078f2b7007df2ef00bd
:101d60007ef2ef001d00370030cbb3007752e30066
:101d700005003a0077d2bf0078f2b7007ff2ef009b
:101d800080f2ef001500370030ccb3007752e3004b
:101d900004003a0077d2bf0078f2b70081f2ef007a
:101da0000e00370030cdb3007752e30004003a0054
:101db00077d2bf0078f2b70082f2ef000700370059
:101dc00030ceb3007752e30004003a0077d2bf0070
:101dd00078f2b70083f2ef0084f2ef0008013700d9
:101de0007852e20002003a00050137000401370092
:101df00030c8b3007852e3000e003a0000e0ef0074
:101e00007952e30003003a0077d2bf0079f2b700bd
:101e1000070037007752ec007af2b70079d2bf00a2
:101e20008752b50001003a008812a90079f2ef004c
:101e3000f300370030c9b3007852e300b4003a0031
:101e400000e0ef007b52e30003003a0077d2bf00ce
:101e50007bf2b700ad00370077d2bf007cf2b7004d
:101e60007c52e20005003a007bd2bf008752b500e9
:101e700001003a008812a900a40037007bd2bf00fd
:101e800071c1b30080cf100025003600d0c2b3006e
:101e90007b52e30022003e002068a9007bd2bf00f5
:101ea0000080fb0000004000e138210060807800e5
:101eb0005092880050928000100888008c52e200f6
:101ec000080036008cd2bf000081fb0050928000d9
:101ed0000200e00002003200110009000280d80078
:101ee000b0928800b0928000c09288005832d5002d
:101ef000d091800040908800e09180005090880050
:101f000040908000609088000068a9002068a800c8
:101f10007bd2bf0087f2b7008812a8007a00370092
:101f20007bd2bf00d1c2b30080cf100025003600a5
:101f3000c0c3b3007b52e30022003e002068a9002a
:101f40007bd2bf000080fb0000004000e138210090
:101f500060807800509288005092800010088800bd
:101f60008c52e200080036008cd2bf000081fb00da
:101f7000509280000200e0000200320011000900cf
:101f80000280d800b0928800b0928000c092880091
:101f90005832d500f0918000409088000092800077
:101fa0005090880040908000609088000068a900f0
:101fb0002068a8007bd2bf0087f2b7008812a80073
:101fc000510037007bd2bf00c1c3b30080cf1000e7
:101fd00025003600d0c4b3007b52e30022003e004f
:101fe0002068a9007bd2bf000080fb0000004000f9
:101ff000e138210060807800509288005092800083
:10200000100888008c52e200080036008cd2bf0015
:102010000081fb00509280000200e00002003200cc
:10202000110009000280d800b0928800b0928000b0
:10203000c09288005832d5001092800040908800ed
:10204000209280005090880040908000609088002e
:102050000068a9002068a8007bd2bf0087f2b70003
:102060008812a800280037007bd2bf00d1c4b3007b
:1020700080cf100024003600a0c5b3007b52e300df
:1020800021003e002068a9007bd2bf000080fb0039
:1020900000004000e1382100608078005092880004
:1020a00050928000100888008c52e2000800360030
:1020b0008cd2bf000081fb00509280000200e00043
:1020c00002003200110009000280d800b09288009e
:1020d000b0928000c09288005832d50030928000c3
:1020e000409088004092800050908800409080008e
:1020f000609088000068a9002068a8007bd2bf001b
:1021000087f2b7008812a8007bf2ef003c0037008e
:1021100030cab3007852e3000a003a0000e0ef0052
:102120007d52e30003003a0077d2bf007df2b70092
:102130000300370077d2bf007ef2b7003f000700f0
:102140002f00370030cbb3007852e3000a003a008a
:1021500000e0ef007f52e30003003a0077d2bf00b7
:102160007ff2b7000300370077d2bf0080f2b700dc
:10217000af0007002200370030ccb3007852e300f4
:1021800009003a0000e0ef008152e30004003a0049
:1021900077d2bf0081f2b7002a00070001003700a4
:1021a00081f2ef001600370030cdb3007852e30023
:1021b00007003a0000e0ef008252e30003003a001b
:1021c00077d2bf0082f2b700970007000c003700fb
:1021d00030ceb3007852e30009003a0000e0ef008f
:1021e0008352e30003003a0077d2bf0083f2b700c6
:1021f0000300370077d2bf0084f2b7001300070056
:102200008c52e20002003a005432ef00080037001e
:102210007bf80700a08f8800b0928000f411b60010
:1022200090928800909280005812b500a092880089
:1022300012aeaa0010aea900a6fe37007df2ef0094
:102240000000060081f2ef00000006008752e20065
:102250007100360084d2bf008552b50001003a00fb
:102260006c00370010c4b3008452b5002e00390052
:1022700084d2bf000080fb0001fc2f000100400061
:102280008092880002002000c327240080928000f2
:10229000a2fa0700e4f907004093880051938800f0
:1022a00087d2bf000080fb0000004000e10823004f
:1022b00060807800a08f88000200200003002400c6
:1022c000a08f800095fa0700d7f90700429380009d
:1022d0005393800017fa07004093880051938800b9
:1022e00040938000519380006cfa07008092880030
:1022f00087d2bf000080fb0000004000e1382100d1
:1023000060807800a08f880080928000f411b50072
:10231000509288005012ee002090880084d2bf00b6
:1023200085f2b7003b00370000c4b3008452e300dd
:102330000b003a005032ef0087d2bf000080fb0054
:1023400000004000e1382100608078005092880051
:102350000432ef0084d2bf0085f2b7002d003700b1
:1023600084d2bf008080fb000004200001005000e8
:1023700080928800020020000328240080928000c0
:1023800066fa0700a8f90700409388005193880077
:1023900087d2bf000080fb0000004000e10823005e
:1023a00060807800a08f88000200200003002400d5
:1023b000a08f800059fa07009bf907004293800024
:1023c00053938000dbf90700409388005193880005
:1023d000409380005193800030fa0700809288007b
:1023e00087d2bf000080fb0000004000e1382100e0
:1023f00060807800a08f880080928000f411b40083
:1024000050928800809280002090880084d2bf0083
:1024100085f2b700020037000432ef0085f2ef00ca
:1024200084f2ef000000060082f2ef0000000600d8
:102430007fd2bf0080407800e1cf500007003a0013
:1024400080d2bf000080fb004206de00e09a23003d
:1024500060407e008cf2b700790137007fd2bf0068
:1024600080407800e3cf500003003a0080d2bf00e4
:1024700089f2b700720137007fd2bf008040780038
:10248000e4cf500009003a0080d2bf008af2b700c2
:102490008ad2bf000080fb0000004000e12821003c
:1024a00060807800d0088800650137007fd2bf00c7
:1024b00080407800f4cf50004e003a002068a90018
:1024c0000068a90000402000306188006cb2ef0075
:1024d0006eb2ef00462cef008772ef00d0c3b3005e
:1024e0008052e30007003a00ec382100e078230036
:1024f0007f000900301e780080d2bf008df2b70047
:102500003b003700e0c3b3008052e30007003a000d
:10251000ec382100e05823007f000900301e7800cd
:1025200080d2bf008df2b70031003700f0c3b30096
:102530008052e30007003a00ec382100e048230015
:102540007f000900301e780080d2bf008df2b700f6
:102550002700370000c4b3008052e30007003a00b0
:10256000ec382100e01823007f000900301e7800bd
:1025700080d2bf008df2b7001d00370010c4b30039
:102580008052e30007003a00ec382100e0282300e5
:102590007f000900301e780080d2bf008df2b700a6
:1025a0001300370020c4b3008052e30007003a0054
:1025b000ec382100e03823007f000900301e78004d
:1025c00080d2bf008df2b7000900370030c4b300dd
:1025d0008052e30006003a00ec382100e068230056
:1025e0007f000900301e780080d2bf008df2b70056
:1025f0001301370080c2b3007f52e3003d003a0070
:102600008052e20005003a00f0908000d0918800ee
:1026100000918000e09188003500370080d2bf0033
:1026200080407800e1cf500005003a001091800012
:10263000d091880020918000e09188002c00370024
:1026400080d2bf0080407800e2cf500005003a0001
:1026500030918000d091880040918000e091880006
:102660002300370080d2bf0080407800e3cf5000c5
:1026700005003a0050918000d09188006091800060
:10268000e09188001a00370080d2bf0080407800b7
:10269000e4cf500005003a0070918000d09188008e
:1026a00080918000e09188001100370080d2bf0047
:1026b00080407800e5cf500005003a0090918000fe
:1026c000d0918800a0918000e09188000800370038
:1026d00080d2bf0080407800e6cf500004003a006e
:1026e000b0918000d0918800c0918000e091880076
:1026f000d300370090c2b3007f52e3003d003a00a0
:102700008052e20005003a00f0908000f0918800cd
:1027100000918000009288003500370080d2bf0011
:1027200080407800e1cf500005003a001091800011
:10273000f091880020918000009288002c003700e2
:1027400080d2bf0080407800e2cf500005003a0000
:1027500030918000f09188004091800000928800c4
:102760002300370080d2bf0080407800e3cf5000c4
:1027700005003a0050918000f0918800609180003f
:10278000009288001a00370080d2bf008040780095
:10279000e4cf500005003a0070918000f09188006d
:1027a00080918000009288001100370080d2bf0025
:1027b00080407800e5cf500005003a0090918000fd
:1027c000f0918800a09180000092880008003700f6
:1027d00080d2bf0080407800e6cf500004003a006d
:1027e000b0918000f0918800c09180000092880034
:1027f00093003700a0c2b3007f52e3003d003a00cf
:102800008052e20005003a00f090800010928800ab
:1028100000918000209288003500370080d2bf00f0
:1028200080407800e1cf500005003a001091800010
:102830001092880020918000209288002c003700a0
:1028400080d2bf0080407800e2cf500005003a00ff
:102850003091800010928800409180002092880082
:102860002300370080d2bf0080407800e3cf5000c3
:1028700005003a005091800010928800609180001d
:10288000209288001a00370080d2bf008040780074
:10289000e4cf500005003a0070918000109288004b
:1028a00080918000209288001100370080d2bf0004
:1028b00080407800e5cf500005003a0090918000fc
:1028c00010928800a09180002092880008003700b4
:1028d00080d2bf0080407800e6cf500004003a006c
:1028e000b091800010928800c091800020928800f2
:1028f00053003700b0c2b3007f52e3003d003a00fe
:102900008052e20005003a00f0908000309288008a
:1029100000918000409288003500370080d2bf00cf
:1029200080407800e1cf500005003a00109180000f
:102930003092880020918000409288002c0037005f
:1029400080d2bf0080407800e2cf500005003a00fe
:102950003091800030928800409180004092880041
:102960002300370080d2bf0080407800e3cf5000c2
:1029700005003a00509180003092880060918000fc
:10298000409288001a00370080d2bf008040780053
:10299000e4cf500005003a0070918000309288002a
:1029a00080918000409288001100370080d2bf00e3
:1029b00080407800e5cf500005003a0090918000fb
:1029c00030928800a0918000409288000800370073
:1029d00080d2bf0080407800e6cf500004003a006b
:1029e000b091800030928800c091800040928800b1
:1029f0001300370020c4b3007f52e30007003a0001
:102a00008052e20002003a000f0007000200370087
:102a1000048ea8003000070009003700b0c7b300db
:102a20007f52e30006003a002068a9000040200021
:102a3000306188008812a9008772ef0085f2ef00ec
:102a40007ff2ef00000006002068a900004020008f
:102a50003061880085f2ef00008ea900048ea90085
:102a60000000370070908000d09188008090800036
:102a7000e091880090908000f0918800a090800004
:102a800000928800b090800010928800c090800072
:102a900020928800d090800030928800e0908000e2
:102aa0004092880000c3b3008cf2b70080c0b3002e
:102ab00089f2b700e0c5b3008af2b700ec38210014
:102ac000e01823007f000900301e780000c4b30026
:102ad0008df2b7000000370089d2bf008080fb0074
:102ae0008ad2bf000080fb000200bc000200e000b0
:102af000090036001421ef000368a9008ad2bf0044
:102b00000080fb0000004000e12821006080780088
:102b1000d00888002368a800000006008eb2ef00ed
:102b2000a0c72500809488005098250090948800c4
:102b300040812500a0948800906a2500b094880008
:102b400030542500c0948800303e2500d094880081
:102b500090282500e094880050132500f094880008
:102b600060fe240000958800c0e9240010958800cc
:102b700080d524002095880090c1240030958800dd
:102b8000f0ad240040958800a09a2400509588005c
:102b9000a087240060958800f07424007095880058
:102ba00090622400809588008050240090958800d1
:102bb000b03e2400a0958800302d2400b0958800f8
:102bc000f01b2400c0958800000b2400d0958800dd
:102bd00050fa2300e0958800e0e92300f095880092
:102be000c0d9230000968800e0c923001096880011
:102bf00040ba230020968800e0aa2300309688007f
:102c0000c09b230040968800e08c230050968800eb
:102c1000307e230060968800d06f23007096880075
:102c2000a061230080968800b0532300909688000e
:102c3000f0452300a096880070382300b0968800e5
:102c4000202b2300c0968800101e2300d0968800f9
:102c500040112300e096880090042300f09688003d
:102c600020f8220000978800e0eb220010978800ef
:102c7000d0df220020978800f0d322003097880010
:102c800050c8220040978800d0bc2200509788008e
:102c900080b122006097880070a62200709788009b
:102ca000809b220080978800c09022009097880027
:102cb00020862200a0978800c07b2200b097880061
:102cc00080712200c097880060672200d09788003a
:102cd000805d2200e0978800c0532200f0978800b2
:102ce000204a220000988800b040220010988800f6
:102cf0006037220020988800402e220030988800fb
:102d00004025220040988800601c220050988800ce
:102d1000b013220060988800200b22007098880071
:102d2000b00222008098880060fa21009098880004
:102d300040f22100a098880030ea2100b098880075
:102d400050e22100c098880090da2100d0988800d5
:102d5000e0d22100e098880060cb2100f098880044
:102d6000f0c3210000998800b0bc210010998800b0
:102d700080b521002099880080ae2100309988001c
:102d800090a7210040998800b0a0210050998800a8
:102d9000009a210060998800609321007099880052
:102da000e08c21008099880080862100909988001d
:102db00030802100a0998800007a2100b099880015
:102dc000f0732100c0998800f06d2100d09988002f
:102dd00000682100e099880040622100f099880095
:102de000805c2100009a8800e0562100109a88003b
:102df00060512100209a8800f04b2100309a880011
:102e000090462100409a880050412100509a880045
:102e1000203c2100609a880010372100709a8800b9
:102e200010322100809a8800202d2100909a88007d
:102e300040282100a09a880080232100b09a8800b1
:102e4000d01e2100c09a8800301a2100d09a880034
:102e5000a0152100e09a880020112100f09a880036
:102e6000c00c2100009b880070082100109b880086
:102e700020042100209b8800f0ff2000309b880068
:102e8000d0fb2000409b8800c0f72000509b8800aa
:102e9000d0f32000609b8800e0ef2000709b88004a
:102ea00000ec2000809b880030e82000909b880088
:102eb00070e42000a09b8800c0e02000b09b880048
:102ec00020dd2000c09b880090d92000d09b880086
:102ed00010d62000e09b8800a0d22000f09b880044
:102ee00040cf2000009c8800e0cb2000109c880090
:102ef000a0c82000209c880060c52000309c88006d
:102f000030c22000409c880010bf2000509c8800e8
:102f100000bc2000609c88000000060010c0b300c8
:102f200086f2b700e0c7b3008652e30022003e00fd
:102f300086d2bf000080fb000006e9000c064600b8
:102f4000e018230060007e00a08f880086d2bf00ba
:102f50000080fb000006e8000c064600e018230095
:102f600060007e00f411b5006128210091407800d6
:102f70008180fb0081804000e208230080307900de
:102f800086d2bf000080fb0000004000e108230063
:102f9000608078004100de006128210091407800c7
:102fa0008180fb0081804000e208230080307900ae
:102fb0008672ec00dbff3900000923001000780066
:102fc000e108230080087800a01823001000780092
:102fd000c11823008008780000000600505020002f
:102fe00070a48800705d200080a48800c04d20007f
:102ff00090a48800504a2000a0a4880080492000a6
:10300000b0a48800804a2000c0a48800b0462000f8
:10301000d0a4880090382000e0a488003038200038
:10302000f0a48800b035200000a58800a021200071
:1030300010a588000013200020a58800200c200087
:1030400030a588002002200040a588004004200010
:1030500050a588005011200060a588001022200093
:1030600070a58800802d200080a58800e038200011
:1030700090a58800e0442000a0a58800904f200083
:10308000b0a5880000542000c0a58800605620002c
:10309000d0a58800a05c2000e0a58800606020002a
:1030a000f0a58800c062200000a6880060622000b1
:1030b00010a68800805f200020a68800f05d200018
:1030c00030a688009059200040a68800a054200017
:1030d00050a688008052200060a688001052200070
:1030e00070a688005053200080a68800e05420007d
:1030f00090a6880090552000a0a68800d0552000fa
:10310000b0a6880060542000c0a68800305420007b
:10311000d0a68800e0522000e0a6880040512000a0
:10312000f0a68800d050200000a78800304c200076
:1031300010a788001048200020a788002046200003
:1031400030a788005040200040a78800403e200063
:1031500050a78800b03f200060a78800a03f200053
:1031600070a788004040200080a78800904320007e
:1031700090a7880000452000a0a78800e044200018
:10318000b0a78800c0462000c0a78800d047200014
:10319000d0a78800b0472000e0a788005047200053
:1031a000f0a788006046200000a88800d0452000d5
:1031b00010a888007044200020a88800c04120008a
:1031c00030a88800c03e200040a88800303e200083
:1031d00050a88800203e200060a88800203c2000e5
:1031e00070a88800803a200080a88800c03b20009a
:1031f00090a88800d03c2000a0a88800c03d2000f6
:10320000b0a88800c03f2000c0a88800304120003e
:10321000d0a8880070422000e0a88800f043200079
:10322000f0a888002044200000a988001045200054
:1032300010a988004045200020a98800a044200053
:1032400030a988007044200040a98800a0442000d4
:1032500050a98800f042200060a98800b0402000fa
:1032600070a98800503f200080a98800f03d200010
:1032700090a98800203c2000a0a98800703a200076
:10328000b0a9880030392000c0a98800c0372000cc
:10329000d0a98800d0362000e0a98800d0362000d0
:1032a000f0a988003037200000aa880040372000ad
:1032b00010aa88006036200020aa880090352000df
:1032c00030aa8800d034200040aa88004034200072
:1032d00050aa88003034200060aa8800a034200062
:1032e00070aa88002035200080aa88008035200040
:1032f00090aa8800a0352000a0aa8800b035200040
:10330000b0aa880010362000c0aa8800b03720007c
:10331000d0aa8800d0382000e0aa880030392000e8
:10332000f0aa8800a037200000ab880040352000bc
:1033300010ab88000034200020ab8800a0332000b0
:1033400030ab88009032200040ab880080312000f4
:1033500050ab88009030200060ab8800802f2000a8
:1033600070ab8800c02e200080ab8800b02d2000fc
:1033700090ab8800a02c2000a0ab8800102d20006e
:10338000b0ab8800902e2000c0ab8800a02f20009a
:10339000d0ab8800a02e2000e0ab8800c02c20001d
:1033a000f0ab8800002e200000ac88002031200007
:1033b00010ac8800a034200020ac8800203620000b
:1033c00030ac88008036200040ac8800f02b200014
:1033d00050ac8800e037200060ac88009057200097
:1033e00070ac8800c059200080ac8800d04b200011
:1033f00090ac8800604b2000a0ac88008048200082
:10340000b0ac8800604a2000c0ac8800c0422000f8
:10341000d0ac880000362000e0ac88005039200095
:10342000f0ac88000035200000ad8800201c200092
:1034300010ad8800a010200020ad8800c009200039
:1034400030ad88003000200040ad8800100720001b
:1034500050ad88002016200060ad8800a023200019
:1034600070ad88009031200080ad8800403d200084
:1034700090ad880070482000a0ad88006051200009
:10348000b0ad880050542000c0ad88000057200027
:10349000d0ad8800505c2000e0ad88006060200066
:1034a000f0ad8800b062200000ae8800906120007e
:1034b00010ae8800105f200020ae8800005d200064
:1034c00030ae88001058200040ae880040542000e4
:1034d00050ae88006052200060ae8800605220002c
:1034e00070ae88001054200080ae88000055200087
:1034f00090ae8800f0552000a0ae8800b0552000a6
:10350000b0ae880010542000c0ae880020542000c7
:10351000d0ae880000522000e0ae880000512000ac
:10352000f0ae88005050200000af8800704a2000a4
:1035300010af8800e046200020af880050452000f2
:1035400030af8800603f200040af8800903e2000f0
:1035500050af8800f03f200060af8800803f20001f
:1035600070af88006041200080af88004044200098
:1035700090af8800e0442000a0af8800b045200054
:10358000b0af880060472000c0af8800904720009f
:10359000d0af8800d0472000e0af8800104720005f
:1035a000f0af8800c045200000b0880080452000b2
:1035b00010b088005044200020b088000041200056
:1035c00030b08800203e200040b08800e03d200060
:1035d00050b08800b03d200060b08800803b2000e3
:1035e00070b08800a03a200080b08800103c200015
:1035f00090b08800003d2000a0b08800d03d2000a1
:10360000b0b0880040402000c0b088004041200099
:10361000d0b0880020422000e0b08800d0432000d5
:10362000f0b088001044200000b18800f044200071
:1036300010b188002045200020b18800a04420005f
:1036400030b188009044200040b1880050442000f0
:1036500050b188008042200060b188009040200076
:1036600070b18800f03e200080b18800903d2000bd
:1036700090b18800a03b2000a0b18800603a2000f3
:10368000b0b1880010392000c0b188008037200018
:10369000d0b1880070362000e0b18800d03620001c
:1036a000f0b188007037200000b288006037200039
:1036b00010b288002036200020b28800203520007b
:1036c00030b28800d034200040b28800403420005e
:1036d00050b288005034200060b28800e0342000ee
:1036e00070b288005035200080b2880080352000fc
:1036f00090b28800f0352000a0b28800d0352000bc
:10370000b0b2880050362000c0b28800f0372000e8
:10371000d0b28800c0382000e0b28800d038200045
:10372000f0b288005037200000b38800a034200099
:1037300010b388008033200020b38800203320009d
:1037400030b388001032200040b38800b030200031
:1037500050b38800e02f200060b38800402f200085
:1037600070b38800c02e200080b38800702d200028
:1037700090b38800902c2000a0b38800602d20001a
:10378000b0b38800602f2000c0b38800c02f200095
:10379000d0b38800002e2000e0b38800d02c200099
:1037a000f0b38800602e200000b48800d0312000e3
:1037b00010b48800d034200020b488006037200086
:1037c00030b488009032200040b48800a027200048
:1037d00050b48800703b200060b48800205e200058
:1037e00070b48800b053200080b48800304b2000b3
:1037f00090b48800804b2000a0b48800404820008e
:10380000b0b48800c04a2000c0b488004041200005
:10381000d0b4880020372000e0b488006039200050
:10382000f0b48800b02e200000b5880050182000a9
:1038300010b58800b00f200020b588009006200049
:1038400030b58800a836ef00c00a200050b58800c7
:10385000f019200060b58800d026200070b58800df
:10386000b034200080b58800c040200090b58800aa
:10387000904a2000a0b5880020512000b0b58800f3
:10388000b0542000c0b58800b0582000d0b58800e2
:10389000605d2000e0b5880070602000f0b5880011
:1038a000c062200000b688007060200010b688005a
:1038b000d05e200020b68800405b200030b6880033
:1038c0005056200040b688006053200050b6880053
:1038d0001052200060b688009052200070b6880018
:1038e0005054200080b68800e054200090b6880034
:1038f00050562000a0b6880010552000b0b68800b1
:1039000020542000c0b6880050542000d0b6880053
:1039100070512000e0b6880010512000f0b68800f9
:10392000404f200000b788008049200010b7880071
:10393000e046200020b78800b043200030b7880060
:10394000203f200040b78800403f200050b788004b
:10395000f03f200060b78800203f200070b788004b
:10396000c041200080b78800d044200090b7880074
:1039700080442000a0b78800c0452000b0b7880070
:10398000f0472000c0b78800d0472000d0b788009b
:1039900070472000e0b78800f0462000f0b78800ac
:1039a0009045200000b888003045200010b88800fd
:1039b000b043200020b88800f03f200030b88800d5
:1039c000d03d200040b88800e03d200050b888007d
:1039d000603d200060b88800803a200070b8880000
:1039e000903a200080b88800003c200090b8880001
:1039f000103d2000a0b88800c03e2000b0b888006c
:103a0000b0402000c0b8880090412000d0b88800a5
:103a100050432000e0b8880080442000f0b88800bf
:103a20007044200000b988002045200010b98800ab
:103a3000b044200020b988006044200030b98800dc
:103a40008044200040b98800b043200050b988006d
:103a5000e041200060b988004040200070b9880033
:103a6000b03e200080b98800e03c200090b988007a
:103a7000003b2000a0b98800d0392000b0b98800f0
:103a8000c0382000c0b9880070372000d0b9880045
:103a9000c0362000e0b9880040372000f0b9880027
:103aa0008037200000ba88000037200010ba880054
:103ab0000036200020ba88001035200030ba880077
:103ac0005034200040ba88009033200050ba88005b
:103ad000b033200060ba8800a034200070ba88009b
:103ae0003035200080ba88005035200090ba880018
:103af000c0352000a0ba8800f0352000b0ba880098
:103b0000e0362000c0ba880040382000d0ba8800d3
:103b100030392000e0ba8800d0382000f0ba8800a0
:103b2000e036200000bb8800c034200010bb8800b5
:103b3000e033200020bb88003033200030bb8800f9
:103b4000f031200040bb8800d030200050bb8800fe
:103b5000a02f200060bb8800e02e200070bb8800f2
:103b6000402e200080bb8800c02c200090bb880025
:103b7000602c2000a0bb8800902d2000b0bb8800e6
:103b8000a02f2000c0bb8800902f2000d0bb880051
:103b9000b02d2000e0bb8800202d2000f0bb880065
:103ba000b02f200000bc88004033200010bc8800eb
:103bb0002035200020bc88006035200030bc880003
:103bc000c032200040bc8800402c200050bc88003f
:103bd000e03f200060bc8800705d200070bc880061
:103be0007051200080bc8800404a200090bc8800b2
:103bf000904b2000a0bc880020482000b0bc88006a
:103c0000004a2000c0bc8800803e2000d0bc880054
:103c1000a0352000e0bc8800e0372000f0bc880020
:103c2000402c200000bd88006018200010bd8800d6
:103c3000b00d200020bd88000006200030bd8800a7
:103c40002001200040bd8800b00d200050bd88003c
:103c5000b01c200060bd8800c029200070bd880015
:103c6000f034200080bd88006042200090bd8800b4
:103c7000204c2000a0bd880080522000b0bd8800ec
:103c800030552000c0bd8800a0592000d0bd88005c
:103c9000705e2000e0bd8800d0602000f0bd88008c
:103ca0009062200000be88001060200010be8800d6
:103cb000505e200020be8800605b200030be88007f
:103cc0008055200040be88001053200050be880060
:103cd0001052200060be8800e052200070be8800b4
:103ce000b054200080be8800f054200090be8800b0
:103cf00000562000a0be8800b0542000b0be88004e
:103d0000f0532000c0be880010542000d0be8800b0
:103d100000512000e0be8800f0502000f0be880076
:103d2000e04e200000bf8800b049200010bf88008e
:103d30003046200020bf88000043200030bf8800ac
:103d4000003f200040bf8800f03e200050bf8800a8
:103d5000d03f200060bf8800e03f200070bf880097
:103d60007042200080bf8800e044200090bf88009f
:103d7000f0442000a0bf880020462000b0bf88008b
:103d800090472000c0bf880090472000d0bf880027
:103d900080472000e0bf880080462000f0bf8800f8
:103da000a045200000c088003045200010c08800d9
:103db0000043200020c08800d03f200030c0880091
:103dc000b03d200040c08800c03d200050c08800a9
:103dd000e03c200060c08800803a200070c088006d
:103de000203b200080c08800703c200090c08800ec
:103df000c03d2000a0c08800303f2000b0c0880037
:103e0000f0402000c0c0880030422000d0c08800b0
:103e100010432000e0c0880040442000f0c088002b
:103e20009044200000c188002045200010c1880077
:103e30009044200020c188004044200030c1880008
:103e4000a044200040c18800d043200050c1880019
:103e5000a041200060c188003040200070c188006f
:103e6000a03e200080c18800e03c200090c1880076
:103e7000703b2000a0c18800f0392000b0c188004c
:103e8000e0382000c0c1880070372000d0c1880011
:103e9000e0362000e0c1880000372000f0c1880033
:103ea0004037200000c28800b036200010c28800d1
:103eb0009035200020c28800f034200030c28800f5
:103ec0003034200040c288009033200050c2880067
:103ed0000034200060c28800b034200070c2880026
:103ee0006035200080c288009035200090c2880094
:103ef000f0352000a0c2880020362000b0c2880023
:103f0000f0362000c0c2880090382000d0c288005f
:103f100090392000e0c2880090382000f0c288006c
:103f20008036200000c388009034200010c3880031
:103f30009033200020c38800f032200030c3880076
:103f40005031200040c388004030200050c388001a
:103f5000402f200060c38800a02e200070c388007e
:103f6000102e200080c38800d02c200090c3880031
:103f7000f02c2000a0c38800302e2000b0c38800a1
:103f8000602f2000c0c38800202f2000d0c38800ed
:103f9000a02d2000e0c38800202d2000f0c3880061
:103fa000602f200000c488008033200010c48800e7
:103fb0006035200020c488007038200030c488009c
:103fc0009029200040c48800302c200050c4880074
:103fd000f03f200060c4880000000600d04a2000a6
:103fe00070c48800d051200080c48800f0452000b3
:103ff00090c48800e0412000a0c48800a0402000b8
:10400000b0c48800403f2000c0c48800a03b20000e
:10401000d0c48800502f2000e0c48800502d20001c
:10402000f0c48800c028200000c58800501a200075
:1040300010c588001010200020c58800e00a20006c
:1040400030c588002003200040c58800b002200051
:1040500050c58800300b200060c588003016200055
:1040600070c58800101e200080c5880040272000f1
:1040700090c58800f0302000a0c58800c03b20001b
:10408000b0c58800a0402000c0c588007043200053
:10409000d0c58800e0462000e0c5880050472000d9
:1040a000f0c58800e048200000c68800e0472000f6
:1040b00010c68800d044200020c68800f0442000ac
:1040c00030c688006045200040c68800c0492000f6
:1040d00050c68800d04a200060c68800304f2000bb
:1040e00070c688009051200080c68800d052200001
:1040f00090c6880060522000a0c68800805320002f
:10410000b0c68800e0552000c0c688006056200078
:10411000d0c68800e0532000e0c68800505220003e
:10412000f0c688007053200000c78800705120003e
:1041300010c788008051200020c78800e05120006f
:1041400030c78800504e200040c78800c04a200079
:1041500050c788006046200060c78800c044200027
:1041600070c788003043200080c78800f0432000db
:1041700090c78800e0412000a0c78800d0412000ff
:10418000b0c78800e0442000c0c788005046200027
:10419000d0c7880040482000e0c7880000492000c0
:1041a000f0c788005048200000c888003042200036
:1041b00010c88800303d200020c88800203720002b
:1041c00030c888000035200040c888003035200005
:1041d00050c888007035200060c888007034200006
:1041e00070c888009033200080c888008037200085
:1041f00090c88800b03a2000a0c88800d03d2000b8
:10420000b0c88800b03e2000c0c88800603e2000d2
:10421000d0c88800903f2000e0c8880020422000dd
:10422000f0c88800e042200000c98800d045200086
:1042300010c98800f046200020c98800b046200040
:1042400030c98800a046200040c98800604720008f
:1042500050c988008047200060c98800b045200010
:1042600070c988009041200080c98800e03e20008d
:1042700090c98800f03a2000a0c988005039200079
:10428000b0c98800c0392000c0c98800d0392000da
:10429000d0c9880060392000e0c98800903820002b
:1042a000f0c988001038200000ca8800f0372000cc
:1042b00010ca88002037200020ca8800a0362000bd
:1042c00030ca88006036200040ca8800803620004e
:1042d00050ca8800b037200060ca8800d03820005b
:1042e00070ca8800f03c200080ca8800803f20000f
:1042f00090ca880040412000a0ca88008040200069
:10430000b0ca880030402000c0ca8800b0422000f7
:10431000d0ca880050442000e0ca88003045200000
:10432000f0ca88001045200000cb8800f04620002d
:1043300010cb88005047200020cb88000048200088
:1043400030cb8800b047200040cb8800f0482000e8
:1043500050cb8800e048200060cb8800b0462000a9
:1043600070cb88006045200080cb8800a0442000ee
:1043700090cb8800c0432000a0cb88005042200092
:10438000b0cb8800c0422000c0cb88001044200081
:10439000d0cb8800b0432000e0cb880060402000f4
:1043a000f0cb8800403f200000cc8800503f200028
:1043b00010cc8800003f200020cc8800a03f2000c7
:1043c00030cc8800203f200040cc8800603720009f
:1043d00050cc8800a03e200060cc8800e053200034
:1043e00070cc88009053200080cc8800f0482000da
:1043f00090cc880070472000a0cc88008045200029
:10440000b0cc880030472000c0cc8800804120001c
:10441000d0cc8800e0362000e0cc8800a038200016
:10442000f0cc88002036200000cd88002025200018
:1044300010cd8800801c200020cd8800f0162000c0
:1044400030cd8800800e200040cd88000012200072
:1044500050cd88001019200060cd88002021200058
:1044600070cd8800102a200080cd8800c031200047
:1044700090cd880040392000a0cd8800203f20004a
:10448000b0cd880020412000c0cd8800f041200040
:10449000d0cd8800c0442000e0cd880090462000a8
:1044a000f0cd8800e047200000ce88007046200054
:1044b00010ce8800b044200020ce88001044200098
:1044c00030ce88007041200040ce8800d0402000cf
:1044d00050ce88004040200060ce8800104120006f
:1044e00070ce8800e041200080ce8800804020000f
:1044f00090ce880070402000a0ce8800d0402000e0
:10450000b0ce880040412000c0ce8800f04420009a
:10451000d0ce880090452000e0ce8800f0462000f4
:10452000f0ce8800a049200000cf8800a0462000df
:1045300010cf88005046200020cf88001046200071
:1045400030cf88009042200040cf8800c04120003a
:1045500050cf8800a041200060cf8800904120000b
:1045600070cf88008045200080cf8800104920004f
:1045700090cf8800c04b2000a0cf8800004d2000c5
:10458000b0cf8800d04d2000c0cf8800404d200023
:10459000d0cf8800504b2000e0cf8800a0492000f9
:1045a000f0cf88003047200000d0880090462000df
:1045b00010d08800f044200020d088004042200025
:1045c00030d088002040200040d08800a04020004b
:1045d00050d08800f040200060d08800a03e20002d
:1045e00070d08800003d200080d08800d03b2000a3
:1045f00090d08800503b2000a0d08800403a200096
:10460000b0d08800703b2000c0d08800403c200023
:10461000d0d08800503d2000e0d08800803f2000ae
:10462000f0d08800c03f200000d1880070402000fa
:1046300010d188009040200020d188002040200028
:1046400030d188001040200040d18800a03f2000d9
:1046500050d18800503e200060d18800603d20008d
:1046600070d18800d03c200080d18800003d20001f
:1046700090d18800503c2000a0d18800f03b200061
:10468000b0d18800503b2000c0d18800c039200044
:10469000d0d1880020372000e0d18800703620007b
:1046a000f0d188002036200000d28800203620007b
:1046b00010d28800d035200020d28800703520002c
:1046c00030d28800b035200040d2880090352000dc
:1046d00050d288003036200060d28800c0362000da
:1046e00070d28800f037200080d28800b0382000d7
:1046f00090d28800a03a2000a0d28800803b200001
:10470000b0d28800003e2000c0d288006040200067
:10471000d0d2880090422000e0d28800b042200031
:10472000f0d288008041200000d388002040200083
:1047300010d388005040200020d3880090422000f1
:1047400030d38800d042200040d38800f0432000be
:1047500050d38800a044200060d3880090462000f9
:1047600070d388001047200080d3880010472000b5
:1047700090d38800d0462000a0d38800b047200006
:10478000b0d38800b0482000c0d3880090462000f5
:10479000d0d3880030442000e0d38800f0412000ce
:1047a000f0d388003042200000d48800204220004e
:1047b00010d488000043200020d48800d04220007c
:1047c00030d48800303e200040d488008032200061
:1047d00050d48800303e200060d48800c0542000af
:1047e00070d48800404b200080d488001044200002
:1047f00090d4880050422000a0d48800803f200040
:10480000b0d48800d03f2000c0d488006038200099
:10481000d0d48800402f2000e0d48800702f2000e2
:10482000f0d488000025200000d588005014200016
:1048300010d58800d00c200020d58800f00520007d
:1048400030d58800a83aef00d006200050d5880067
:10485000b010200060d588000019200070d58800b5
:104860005022200080d58800c02b200090d58800e1
:1048700090362000a0d58800403d2000b0d58800ab
:1048800080422000c0d5880040452000d0d5880057
:1048900080472000e0d5880060472000f0d58800e0
:1048a000f048200000d688003048200010d688004c
:1048b000d046200020d688007044200030d68800e2
:1048c000c042200040d68800a046200050d6880074
:1048d000c048200060d68800e04e200070d68800d6
:1048e0005052200080d688004053200090d6880087
:1048f00080532000a0d68800f0532000b0d6880056
:1049000010552000c0d6880020562000d0d6880040
:1049100040532000e0d6880080522000f0d6880066
:10492000e051200000d788002050200010d78800d8
:10493000e04f200020d78800904f200030d788001b
:10494000a04e200040d78800204d200050d788007e
:10495000c047200060d788005045200070d78800ed
:104960008044200080d78800f044200090d7880041
:10497000f0412000a0d7880080422000b0d78800f6
:1049800020452000c0d7880090452000d0d788005f
:10499000f0462000e0d78800a0472000f0d788002c
:1049a0001046200000d88800d042200010d888008f
:1049b000e03a200020d88800d036200030d8880087
:1049c000c034200040d888009034200050d888009f
:1049d0001034200060d888000032200070d8880091
:1049e0008032200080d888009035200090d8880040
:1049f00070392000a0d88800503e2000b0d8880030
:104a0000a03f2000c0d88800103f2000d0d88800e8
:104a100040402000e0d8880020422000f0d88800e4
:104a2000b042200000d988002045200010d988001d
:104a30003046200020d98800e046200030d9880088
:104a40000047200040d98800e047200050d9880066
:104a5000a047200060d988007045200070d98800e8
:104a60008042200080d98800403e200090d98800f4
:104a7000c03b2000a0d98800b0392000b0d9880000
:104a800020392000c0d9880070392000d0d9880092
:104a9000f0382000e0d98800d0382000f0d9880014
:104aa0003038200000da8800a037200010da8800b3
:104ab000e036200020da88007036200030da8800e6
:104ac000f035200040da8800f035200050da880008
:104ad0004037200060da88006038200070da8800f3
:104ae000203b200080da8800703d200090da8800aa
:104af00050402000a0da880060402000b0da880032
:104b000060412000c0da880040432000d0da8800ed
:104b1000d0442000e0da880070442000f0da8800f9
:104b2000b044200000db88000045200010db880036
:104b30006047200020db88008047200030db8800b1
:104b40008047200040db88009047200050db880031
:104b50007047200060db88003046200070db880052
:104b60003045200080db88002045200090db880055
:104b700000452000a0db880010432000b0db880047
:104b800010432000c0db8800b0432000d0db880049
:104b900040432000e0db880060412000f0db88001b
:104ba0004041200000dc88008040200010dc8800ac
:104bb000c040200020dc8800d03e200030dc88008f
:104bc000003c200040dc88003037200050dc8800aa
:104bd000f044200060dc88004058200070dc880031
:104be000a04e200080dc88000047200090dc880078
:104bf00060472000a0dc880000452000b0dc880071
:104c000050462000c0dc8800203e2000d0dc880018
:104c100080362000e0dc8800d0372000f0dc8800ff
:104c20008030200000dd8800a022200010dd8800f8
:104c3000201a200020dd8800a014200030dd88002c
:104c4000e00f200040dd88000017200050dd8800c4
:104c5000d01d200060dd88006025200070dd880008
:104c6000a02b200080dd8800d034200090dd88005b
:104c7000903b2000a0dd880000402000b0dd8800cf
:104c800070412000c0dd8800b0432000d0dd8800e6
:104c900030452000e0dd880040462000f0dd88003f
:104ca000a046200000de8800a044200010de88001e
:104cb0009043200020de8800e042200030de8800a3
:104cc000803f200040de8800903f200050de8800ba
:104cd0003040200060de88007042200070de8800d6
:104ce000b043200080de88007042200090de880003
:104cf000a0422000a0de8800b0412000b0de880085
:104d000010422000c0de8800c0442000d0de8800b1
:104d100020442000e0de8800f0472000f0de88001c
:104d20001048200000df8800d046200010df8800f7
:104d3000b045200020df8800c044200030df88001c
:104d4000c041200040df8800c040200050df8800c4
:104d50002041200060df88007042200070df880062
:104d60004045200080df88000048200090df880058
:104d7000504a2000a0df8800704c2000b0df88007f
:104d8000504e2000c0df8800a04d2000d0df8800fa
:104d9000704b2000e0df8800d0492000f0df880061
:104da000e046200000e08800b045200010e08800c8
:104db0005043200020e088002041200030e088009f
:104dc0005040200040e08800c040200050e08800b3
:104dd0005040200060e08800103e200070e0880015
:104de000103d200080e08800403d200090e08800d9
:104df000203c2000a0e08800203c2000b0e088009b
:104e0000603c2000c0e08800403d2000d0e08800e9
:104e1000103e2000e0e0880000402000f0e0880024
:104e2000b040200000e188000042200010e188002e
:104e30008041200020e188006040200030e18800af
:104e40005040200040e18800403f200050e18800b1
:104e5000503d200060e18800e03b200070e18800c8
:104e6000303b200080e18800303b200090e188004a
:104e7000c03a2000a0e18800803a2000b0e188001c
:104e8000303a2000c0e18800e0382000d0e18800fe
:104e9000a0372000e0e1880020362000f0e1880003
:104ea000f035200000e288007035200010e2880014
:104eb000c034200020e288003035200030e2880035
:104ec0001035200040e288001035200050e28800b4
:104ed0003036200060e288001037200070e2880041
:104ee0007038200080e288000039200090e28800bd
:104ef000803a2000a0e28800903b2000b0e28800c9
:104f0000603e2000c0e2880060402000d0e28800bf
:104f100060422000e0e2880000422000f0e28800c9
:104f20009040200000e38800c03f200010e388008c
:104f30002041200020e38800e041200030e3880089
:104f40008042200040e38800d042200050e38800e7
:104f50009044200060e388008045200070e38800d2
:104f60004047200080e388001047200090e388003d
:104f700010482000a0e38800e0482000b0e388004b
:104f800020492000c0e3880040462000d0e388008c
:104f900000442000e0e38800d0412000f0e38800d6
:104fa000a042200000e488007043200010e4880044
:104fb000d043200020e488000044200030e4880032
:104fc0004038200040e48800e035200050e48800ac
:104fd000f03f200060e4880000000600304120001f
:104fe00070e48800b042200080e4880090422000f5
:104ff00090e4880040422000a0e488002042200085
:10500000b0e4880030412000c0e48800e040200087
:10501000d0e48800f0402000e0e4880080402000d8
:10502000f0e48800b042200000e588000044200041
:1050300010e58800d045200020e58800a04b200026
:1050400030e58800a04e200040e58800e0582000b0
:1050500050e58800a05e200060e58800906920008f
:1050600070e58800906d200080e588006075200064
:1050700090e58800e0782000a0e58800807c200092
:10508000b0e58800207e2000c0e58800f07f200089
:10509000d0e58800b07f2000e0e58800507c20004b
:1050a000f0e588008079200000e68800707020001c
:1050b00010e68800506b200020e68800505e20003b
:1050c00030e68800a057200040e68800905020007d
:1050d00050e68800b04f200060e688006052200053
:1050e00070e68800405c200080e68800005f2000b9
:1050f00090e68800805e2000a0e68800105d200019
:10510000b0e6880080592000c0e6880000582000e2
:10511000d0e6880010512000e0e68800104b200007
:10512000f0e688002044200000e78800704120005d
:1051300010e78800503f200020e78800b03d2000a5
:1051400030e788006039200040e788007038200090
:1051500050e788007035200060e788006034200048
:1051600070e78800d02f200080e78800702c200096
:1051700090e78800b0292000a0e788007027200071
:10518000b0e7880030272000c0e7880040272000d3
:10519000d0e78800a0272000e0e78800e026200074
:1051a000f0e788003025200000e88800801f2000fc
:1051b00010e88800d01c200020e88800801a200019
:1051c00030e88800c019200040e88800401a20001c
:1051d00050e88800e017200060e88800f015200003
:1051e00070e88800a016200080e88800f0172000f2
:1051f00090e8880060172000a0e88800b016200022
:10520000b0e88800e0172000c0e88800601a20009d
:10521000d0e88800001c2000e0e88800801d200005
:10522000f0e888008023200000e98800a025200005
:1052300010e98800402c200020e98800702f200011
:1052400030e98800d035200040e98800503820003f
:1052500050e98800903b200060e98800a03d2000d4
:1052600070e98800e03d200080e98800403e200091
:1052700090e98800a03f2000a0e9880010412000ac
:10528000b0e9880060412000c0e98800904020001b
:10529000d0e9880000412000e0e98800704020004b
:1052a000f0e98800f03f200000ea8800104020006c
:1052b00010ea8800003f200020ea8800703f2000ac
:1052c00030ea8800d03f200040ea880010402000eb
:1052d00050ea88004040200060ea8800303f20000b
:1052e00070ea8800a03f200080ea8800d0402000bb
:1052f00090ea880010412000a0ea880010412000b8
:10530000b0ea880010422000c0ea8800f043200084
:10531000d0ea880010442000e0ea880050422000d3
:10532000f0ea8800b041200000eb8800b041200086
:1053300010eb88001041200020eb8800803e200008
:1053400030eb8800303d200040eb8800f039200031
:1053500050eb8800f037200060eb8800d03520004b
:1053600070eb88002033200080eb8800b0322000f2
:1053700090eb8800a0302000a0eb8800c02f200018
:10538000b0eb8800902e2000c0eb8800c02e2000db
:10539000d0eb880070312000e0eb8800b0312000b5
:1053a000f0eb88007032200000ec880040332000d1
:1053b00010ec8800b036200020ec88007038200007
:1053c00030ec8800003b200040ec8800603c20006e
:1053d00050ec8800d03f200060ec88008041200025
:1053e00070ec8800b042200080ec88004042200031
:1053f00090ec880020422000a0ec8800f0412000c2
:10540000b0ec880080412000c0ec8800d040200033
:10541000d0ec880030412000e0ec8800f040200013
:10542000f0ec88000042200000ed880000452000dc
:1054300010ed88002047200020ed8800204d20003e
:1054400030ed8800a050200040ed8800105b200067
:1054500050ed8800a060200060ed8800106b2000f7
:1054600070ed8800e06e200080ed8800407620001e
:1054700090ed8800f0782000a0ed8800207c2000ce
:10548000b0ed8800707d2000c0ed8800907e200087
:10549000d0ed8800107e2000e0ed8800807a2000aa
:1054a000f0ed88007077200000ee8800f072200098
:1054b00010ee88004069200020ee88001063200074
:1054c00030ee8800d056200040ee880020532000a7
:1054d00050ee88006051200060ee8800c05420002b
:1054e00070ee8800305d200080ee8800b05f200004
:1054f00090ee8800f05e2000a0ee8800405d200065
:10550000b0ee880060592000c0ee8800e05720000f
:10551000d0ee8800704f2000e0ee8800c0492000e7
:10552000f0ee88003043200000ef8800a04020000b
:1055300010ef8800803e200020ef8800603c2000b3
:1055400030ef88009038200040ef8800403720007e
:1055500050ef88005035200060ef88005033200065
:1055600070ef8800b031200080ef8800902b200081
:1055700090ef880040292000a0ef8800a02720009d
:10558000b0ef880070272000c0ef8800c0272000ff
:10559000d0ef880030282000e0ef8800602620004f
:1055a000f0ef8800c024200000f08800601f200079
:1055b00010f08800e01c200020f08800b01a2000c5
:1055c00030f08800101a200040f08800e019200018
:1055d00050f088003017200060f08800a0162000ee
:1055e00070f088008017200080f0880030182000bc
:1055f00090f08800d0162000a0f0880060162000ef
:10560000b0f0880070182000c0f088004019200019
:10561000d0f08800b01c2000e0f08800701e200050
:10562000f0f08800b024200000f1880090262000cf
:1056300010f18800702d200020f18800b03020008b
:1056400030f18800c036200040f18800e0382000aa
:1056500050f18800303c200060f18800b03d20000f
:1056600070f18800d03d200080f18800803e20004d
:1056700090f18800f03f2000a0f1880080412000d8
:10568000b0f18800f0402000c0f188007040200098
:10569000d0f18800e0402000e0f188009040200038
:1056a000f0f188004040200000f2880030402000e7
:1056b00010f28800603f200020f28800c03f2000e8
:1056c00030f288001040200040f288006040200046
:1056d00050f288006040200060f28800c03f200047
:1056e00070f288007040200080f288001041200095
:1056f00090f2880030412000a0f28800a0412000f4
:10570000b0f28800a0422000c0f288009043200040
:10571000d0f2880090432000e0f288002042200070
:10572000f0f28800d041200000f388007041200092
:1057300010f38800a040200020f38800703f200074
:1057400030f38800003d200040f38800403b2000fb
:1057500050f388005037200060f388003035200077
:1057600070f388005032200080f38800c0312000a0
:1057700090f38800d02f2000a0f38800402f200055
:10578000b0f38800702e2000c0f38800302f200076
:10579000d0f3880070312000e0f38800d031200081
:1057a000f0f38800d032200000f48800e0332000bd
:1057b00010f488003037200020f48800c038200022
:1057c00030f48800803b200040f48800203d200019
:1057d00050f488006040200060f48800e041200020
:1057e00070f48800a042200080f48800104220005d
:1057f00090f4880010422000a0f48800d0412000de
:10580000b0f4880020412000c0f48800f04020005f
:10581000d0f4880070412000e0f48800504120005e
:10582000f0f48800c042200000f58800d045200038
:1058300010f588005048200020f58800704e2000a8
:1058400030f588005052200040f58800105d20009f
:1058500050f58800b062200060f58800606c200080
:1058600070f58800f06f200080f5880040772000f8
:1058700090f58800e0792000a0f58800607b20008a
:10588000b0f58800307e2000c0f58800207f200021
:10589000d0f58800707e2000e0f58800b07c200004
:1058a000f0f588009077200000f688000073200053
:1058b00010f68800d068200020f6880000622000e2
:1058c00030f68800c055200040f68800a052200025
:1058d00050f688002051200060f68800e054200037
:1058e00070f68800e05c200080f68800105f2000e1
:1058f00090f68800e05d2000a0f68800905c200013
:10590000b0f6880030582000c0f68800e05620002d
:10591000d0f68800d04d2000e0f6880080482000b6
:10592000f0f688008045200000f7880050402000f5
:1059300010f78800603f200020f78800403c2000de
:1059400030f78800c039200040f78800b0372000c9
:1059500050f78800f035200060f78800b033200051
:1059600070f78800f031200080f78800c02b2000fd
:1059700090f7880010292000a0f7880070272000e9
:10598000b0f7880030272000c0f78800c02620002c
:10599000d0f7880040272000e0f78800e0242000ae
:1059a000f0f78800d022200000f88800901d200029
:1059b00010f88800801b200020f88800d0192000f3
:1059c00030f888008019200040f88800001a200074
:1059d00050f888004016200060f88800f01520007c
:1059e00070f888000018200080f88800d018200087
:1059f00090f8880040182000a0f888003018200097
:105a0000b0f88800301a2000c0f88800e01a2000a2
:105a1000d0f88800501d2000e0f88800801f20008a
:105a2000f0f888001025200000f98800802620006a
:105a300010f98800b02d200020f9880000312000e6
:105a400030f988003037200040f98800f038200015
:105a500050f98800403c200060f98800a03d2000fb
:105a600070f98800803d200080f98800003f200008
:105a700090f98800e03f2000a0f98800c041200094
:105a8000b0f98800c0412000c0f988002041200002
:105a9000d0f98800a0412000e0f9880010412000e2
:105aa000f0f988002041200000fa8800c040200062
:105ab00010fa88003040200020fa88008040200042
:105ac00030fa88004040200040fa880070402000f2
:105ad00050fa88005040200060fa8800703f200093
:105ae00070fa88007040200080fa88004041200051
:105af00090fa880060412000a0fa880060422000ef
:105b0000b0fa880070432000c0fa880040442000aa
:105b1000d0fa880000442000e0fa8800904320007a
:105b2000f0fa8800c042200000fb8800c04220003c
:105b300010fb88003041200020fb8800e03f20005f
:105b400030fb8800803d200040fb8800703b200037
:105b500050fb88001037200060fb8800e0342000f4
:105b600070fb88002032200080fb8800503120002c
:105b700090fb8800e02e2000a0fb8800802e2000f3
:105b8000b0fb8800502d2000c0fb8800702e200044
:105b9000d0fb880040302000e0fb880070302000ff
:105ba000f0fb88004032200000fc880060332000b9
:105bb00010fc8800e034200020fc8800e038200041
:105bc00030fc8800603a200040fc8800d03d200076
:105bd00050fc8800a03f200060fc8800d0422000dc
:105be00070fc88007043200080fc8800e0422000a8
:105bf00090fc8800e0422000a0fc88004042200089
:105c0000b0fc8800b0412000c0fc8800904120001a
:105c1000d0fc8800e0412000e0fc8800e04120004a
:105c2000f0fc88005043200000fd880090462000d2
:105c300010fd88007049200020fd8800c04f200022
:105c400030fd8800b053200040fd8800905e2000a9
:105c500050fd8800f063200060fd8800206920006e
:105c600070fd8800d070200080fd880060742000e6
:105c700090fd8800807a2000a0fd8800e07b200055
:105c8000b0fd8800707e2000c0fd8800407f2000ad
:105c9000d0fd8800607e2000e0fd8800f07c2000c0
:105ca000f0fd88000077200000fe88009072200040
:105cb00010fe88002068200020fe8800306120004f
:105cc00030fe88007055200040fe88009052200071
:105cd00050fe88003052200060fe880050562000a0
:105ce00070fe8800505e200080fe8800506020001a
:105cf00090fe880050602000a0fe8800305d2000eb
:105d0000b0fe8800d05a2000c0fe880060572000f6
:105d1000d0fe880050532000e0fe8800d0472000cd
:105d2000f0fe8800b044200000ff8800a03f200063
:105d300010ff8800d03e200020ff8800003b20009c
:105d400030ff88001039200040ff88008036200096
:105d500050ff8800b034200060ff8800903220009f
:105d600070ff8800d030200080ff8800702a20005b
:105d700090ff8800c0272000a0ff8800b0262000e8
:105d8000b0ff8800a0262000c0ff8800b0262000b9
:105d9000d0ff880030272000e0ff88003026200058
:105da000f0ff880080222000010022008008780097
:105db000402020002100220080087800b01b200035
:105dc0004100220080087800b01a20006100220003
:105dd0008008780070192000810022008008780077
:105de00070192000a100220080087800d015200042
:105df000c10022008008780070162000e100220017
:105e00008008780010192000010122008008780025
:105e1000d01920002101220080087800f01720000e
:105e20004101220080087800001820006101220052
:105e300080087800201b2000810122008008780063
:105e4000901b2000a101220080087800801d200006
:105e5000c101220080087800f01f2000e10122002b
:105e600080087800002520000102220080087800c8
:105e7000102720002102220080087800702e2000c8
:105e80004102220080087800703120006102220067
:105e90008008780080342000810222008008780089
:105ea000e0382000a102220080087800b03a2000eb
:105eb000c102220080087800e03d2000e1022200bb
:105ec00080087800703d20000103220080087800df
:105ed000303f20002103220080087800e03f2000ae
:105ee0004103220080087800a041200061032200c5
:105ef000800878007041200081032200800878002b
:105f000070412000a1032200800878002042200078
:105f1000c10322008008780040422000e1032200f3
:105f20008008780050422000010422008008780098
:105f3000204120002104220080087800e040200059
:105f40004104220080087800804120006104220082
:105f50008008780000412000810422008008780039
:105f6000f0402000a10422008008780000412000b9
:105f7000c10422008008780080402000e104220053
:105f800080087800c04120000105220080087800c8
:105f9000f0412000210522008008780010422000f6
:105fa000410522008008780070422000610522002f
:105fb00080087800f04320008105220080087800e6
:105fc00060442000a105220080087800f0432000f2
:105fd000c105220080087800a0432000e1052200ce
:105fe00080087800c0422000010622008008780066
:105ff000804220002106220080087800b040200066
:106000004106220080087800b03f2000610622008f
:1060100080087800203d200081062200800878005a
:10602000e03a2000a10622008008780070362000a7
:10603000c10622008008780050342000e1062200ca
:1060400080087800c0312000010722008008780015
:10605000d03020002107220080087800702e200018
:106060004107220080087800002e200061072200ee
:1060700080087800502d20008107220080087800d9
:10608000102f2000a1072200800878005030200047
:10609000c107220080087800b0302000e10722000c
:1060a00080087800903120000108220080087800e4
:1060b000d0332000210822008008780050352000cd
:1060c0004108220080087800b038200061082200d2
:1060d00080087800303a200081082200800878008b
:1060e000403e2000a108220080087800f03f2000f8
:1060f000c1082200800878000000060070412000de
:10610000e108220080087800b04420000109220044
:1061100080087800a04a2000210922008008780029
:10612000c05120004109220080087800205620003c
:106130006109220080087800705f20008109220038
:1061400080087800206a2000a109220080087800d9
:1061500010722000c109220080087800907b200086
:10616000e109220080087800607e2000010a2200f8
:1061700080087800707d2000210a220080087800c5
:10618000a0782000410a220080087800d078200002
:10619000610a22008008780000762000810a22002f
:1061a0008008780040762000a10a2200800878004c
:1061b000e0732000c10a220080087800e06e200011
:1061c000e10a220080087800306b2000010b2200d9
:1061d0008008780000682000210b220080087800e9
:1061e00040672000410b220080087800b063200047
:1061f000610b220080087800205f2000810b2200c4
:1062000080087800c0572000a10b22008008780089
:10621000f0542000c10b220080087800405020007c
:10622000e10b220080087800204b2000010c2200a6
:1062300080087800b0462000210c220080087800f9
:10624000603b2000410c22008008780000302000d4
:10625000610c22008008780010292000810c2200a7
:1062600080087800f0242000a10c2200800878002b
:1062700040232000c10c2200800878002024200048
:10628000e10c220080087800a0232000010d2200ec
:106290008008780060222000210d2200800878000c
:1062a000a0232000410d220080087800c025200096
:1062b000610d22008008780010292000810d220045
:1062c00080087800602b2000a10d22008008780053
:1062d000b02c2000c10d220080087800f02c200096
:1062e000e10d220080087800d02b2000010e220052
:1062f00080087800702a2000210e22008008780093
:10630000b0282000410e220080087800502620008e
:10631000610e22008008780050242000810e2200a7
:1063200080087800d0222000a10e2200800878008a
:1063300060222000c10e2200800878000023200087
:10634000e10e22008008780000242000010f2200c6
:106350008008780040252000210f22008008780066
:10636000f0262000410f22008008780050292000ec
:10637000610f220080087800402b2000810f22004e
:1063800080087800f02f2000a10f220080087800fc
:10639000d0332000c10f220080087800f0362000a2
:1063a000e10f220080087800c03a2000011022008e
:1063b00080087800f03c200021102200800878003e
:1063c000303e20004110220080087800104020005c
:1063d0006110220080087800803f20008110220098
:1063e00080087800f03e2000a1102200800878008c
:1063f000603e2000c110220080087800103c200080
:10640000e110220080087800903a2000011122005b
:106410008008780090382000211122008008780040
:10642000f0352000411122008008780070332000f0
:106430006111220080087800c03020008111220004
:1064400080087800102e2000a1112200800878001a
:10645000302d2000c111220080087800902c2000ef
:10646000e111220080087800802c20000112220017
:1064700080087800a02c20002112220080087800db
:10648000d02c20004112220080087800102e20001d
:1064900061122200800878008030200081122200e2
:1064a0008008780070342000a11222008008780053
:1064b00040382000c112220080087800e03a200015
:1064c000e1122200800878003040200001132200f1
:1064d00080087800e0442000211322008008780022
:1064e000904720004113220080087800504b200084
:1064f0006113220080087800a04e20008113220042
:1065000080087800c0502000a11322008008780085
:10651000d0522000c11322008008780020542000af
:10652000e11322008008780020542000011422008a
:1065300080087800a05320002114220080087800f1
:10654000405320004114220080087800705220003f
:106550006114220080087800c050200081142200bd
:1065600080087800a04f2000a11422008008780045
:10657000b04d2000c114220080087800a04c2000fb
:10658000e114220080087800404a20000115220012
:10659000800878002049200021152200800878001a
:1065a000b047200041152200800878006045200097
:1065b0006115220080087800204520008115220006
:1065c0008008780070442000a1152200800878001f
:1065d00000442000c115220080087800604220009d
:1065e000e11522008008780090402000011622006a
:1065f00080087800603d2000211622008008780085
:10660000c03a2000411622008008780000372000a0
:106610006116220080087800a03220008116220036
:106620008008780030312000a11622008008780010
:10663000b02d2000c116220080087800302b2000e9
:10664000e116220080087800302a2000011722007d
:1066500080087800a02820002117220080087800f8
:10666000b0282000411722008008780090282000e0
:10667000611722008008780040292000811722003d
:1066800080087800f0292000a117220080087800f7
:10669000d02b2000c117220080087800402d200058
:1066a000e117220080087800f02e20000118220057
:1066b000800878001031200021182200800878001e
:1066c000f03220004118220080087800f0342000c9
:1066d0006118220080087800c0382000811822004c
:1066e00080087800903b2000a118220080087800e4
:1066f000603f2000c118220080087800004320007d
:10670000e11822008008780040452000011922008d
:106710008008780080492000211922008008780034
:10672000b0512000411922008008780060572000f5
:106730006119220080087800b061200081192200d0
:1067400080087800806b2000a11922008008780062
:1067500070722000c119220080087800e07a2000c1
:10676000e119220080087800a07d2000011a220093
:1067700080087800807d2000211a2200800878009f
:10678000d0792000411a220080087800607a200029
:10679000611a220080087800c0762000811a220049
:1067a0008008780080752000a11a220080087800f7
:1067b00080732000c11a220080087800006e20003b
:1067c000e11a220080087800806d2000011b220061
:1067d00080087800f0682000211b220080087800e3
:1067e00070662000411b220080087800b062200003
:1067f000611b220080087800405e2000811b22007f
:106800008008780090582000a11b220080087800a2
:1068100000562000c11b2200800878003050200064
:10682000e11b22008008780090482000011c220013
:1068300080087800e0422000211c220080087800b7
:1068400060352000411c220080087800402e200086
:10685000611c220080087800a0252000811c2200f5
:106860008008780050242000a11c220080087800b5
:10687000d0232000c11c220080087800d0232000f3
:10688000e11c22008008780010232000011d220056
:106890008008780010222000211d22008008780046
:1068a00020242000411d22008008780000262000be
:1068b000611d220080087800b02b2000811d22007d
:1068c00080087800202d2000a11d2200800878007b
:1068d000a02d2000c11d220080087800c02d2000be
:1068e000e11d220080087800002c2000011e2200fb
:1068f00080087800302b2000211e220080087800bc
:10690000d0282000411e220080087800b0252000f9
:10691000611e22008008780020232000811e2200b2
:1069200080087800d0212000a11e22008008780075
:1069300030212000c11e2200800878004022200063
:10694000e11e22008008780050232000011f220051
:1069500080087800a0242000211f220080087800f1
:10696000a0262000411f220080087800d0292000a6
:10697000611f220080087800402b2000811f220028
:106980008008780030302000a11f220080087800a5
:1069900040332000c11f22008008780060372000ab
:1069a000e11f220080087800403b200001202200e7
:1069b00080087800903d2000212022008008780087
:1069c000303e20004120220080087800103f200047
:1069d0006120220080087800f03f20008120220002
:1069e00080087800803f2000a120220080087800e5
:1069f000a03e2000c120220080087800503d2000e9
:106a0000e120220080087800203b200001212200a4
:106a100080087800103a20002121220080087800a8
:106a200050362000412122008008780000332000e9
:106a3000612122008008780000302000812122009e
:106a400080087800b02d2000a12122008008780065
:106a5000702c2000c121220080087800202c20000a
:106a6000e121220080087800f02b20000122220082
:106a700080087800502b2000212222008008780016
:106a8000d02c20004122220080087800a02f200076
:106a9000612222008008780030322000812222000a
:106aa00080087800b0352000a122220080087800fc
:106ab00090382000c122220080087800f03b20009e
:106ac000e12222008008780090402000012322006b
:106ad00080087800a045200021232200800878004b
:106ae000104920004123220080087800f04c20004b
:106af0006123220080087800204f2000812322009b
:106b000080087800d0512000a1232200800878005e
:106b1000c0532000c1232200800878006054200068
:106b2000e1232200800878009054200001242200f4
:106b300080087800e053200021242200800878009b
:106b4000105320004124220080087800305120009a
:106b50006124220080087800304f20008124220028
:106b600080087800c04e2000a12422008008780010
:106b7000204d2000c124220080087800204c2000f5
:106b8000e124220080087800c0492000012522006d
:106b900080087800a0472000212522008008780086
:106ba000b0462000412522008008780020462000c1
:106bb0006125220080087800704520008125220090
:106bc0008008780080442000a125220080087800f9
:106bd000b0422000c125220080087800004120003a
:106be000e125220080087800503f20000126220085
:106bf00080087800003d20002126220080087800cf
:106c0000c03b20004126220080087800a0362000ea
:106c100061262200800878001032200081262200a0
:106c200080087800802f2000a126220080087800ac
:106c3000b02c2000c126220080087800b02b200054
:106c4000e126220080087800f02920000127220098
:106c50008008780060292000212722008008780021
:106c600030292000412722008008780000292000d8
:106c70006127220080087800702a200081272200e6
:106c800080087800a02a2000a12722008008780030
:106c9000102c2000c127220080087800a02d2000a1
:106ca000e127220080087800902f20000128220090
:106cb00080087800c0312000212822008008780058
:106cc000e03220004128220080087800b035200002
:106cd00061282200800878001038200081282200d6
:106ce00080087800f03a2000a1282200800878006f
:106cf000a03f2000c12822008008780070432000b7
:106d0000e128220080087800604620000129220046
:106d100080087800204b200021292200800878007c
:106d2000e05120004129220080087800905720007f
:106d30006129220080087800f0602000812922006b
:106d400080087800b0692000a1292200800878001e
:106d500030742000c129220080087800a07c200027
:106d6000e129220080087800f07f2000012a22001b
:106d700080087800e07c2000212a2200800878002a
:106d800000772000412a2200800878004079200006
:106d9000612a22008008780090762000812a220053
:106da00080087800f0772000a12a2200800878006f
:106db000d0752000c12a220080087800f06e2000e3
:106dc000e12a220080087800e06d2000012b2200db
:106dd00080087800f0682000212b220080087800cd
:106de00030672000412b220080087800606320007b
:106df000612b220080087800f05e2000812b2200a9
:106e00008008780010592000a12b2200800878000b
:106e1000a0552000c12b220080087800904e200051
:106e2000e12b22008008780080492000012c2200fc
:106e300080087800d03f2000212c220080087800b4
:106e400010322000412c220080087800202b2000e6
:106e5000612c22008008780040242000812c220030
:106e600080087800e0232000a12c22008008780010
:106e7000f0232000c12c220080087800602420002c
:106e8000e12c22008008780000232000012d220040
:106e90008008780010232000212d2200800878002f
:106ea00060262000412d220080087800b0282000b4
:106eb000612d220080087800602d2000812d2200a5
:106ec00080087800f02d2000a12d22008008780095
:106ed000102f2000c12d220080087800f02d200006
:106ee000e12d220080087800e02c2000012e2200f5
:106ef00080087800702b2000212e22008008780066
:106f0000b0272000412e22008008780000262000b3
:106f1000612e22008008780000222000812e2200ad
:106f200080087800e0202000a12e22008008780050
:106f300020202000c12e220080087800302120006f
:106f4000e12e220080087800e0222000012f22009c
:106f50008008780040242000212f2200800878003b
:106f600000262000412f22008008780020292000e0
:106f7000612f220080087800902a2000812f2200b3
:106f800080087800b0302000a12f2200800878000f
:106f900030332000c12f220080087800e038200024
:106fa000e12f220080087800303c200001302200d0
:106fb00080087800c03d2000213022008008780041
:106fc000603f20004130220080087800704020009f
:106fd00061302200800878000041200081302200ca
:106fe00080087800a03f2000a130220080087800af
:106ff000f03f2000c130220080087800903d200042
:10700000e130220080087800503a2000013122004f
:107010008008780070382000213122008008780034
:107020008034200041312200800878004032200066
:107030006131220080087800b030200081312200c8
:1070400080087800d02e2000a1312200800878002e
:10705000f02c2000c131220080087800502c200044
:10706000e131220080087800a02b200001322200ac
:1070700080087800b02b20002132220080087800a0
:10708000f02c20004132220080087800b02f200030
:1070900061322200800878007032200081322200a4
:1070a00080087800b0352000a132220080087800e6
:1070b000b0392000c132220080087800303d200025
:1070c000e132220080087800d04120000133220004
:1070d00080087800d0442000213322008008780006
:1070e000e04820004133220080087800404d200015
:1070f0006133220080087800a04f200081332200f5
:1071000080087800c0522000a13322008008780057
:1071100070542000c1332200800878007054200091
:10712000e1332200800878006054200001342200fe
:107130008008780060532000213422008008780005
:10714000c0522000413422008008780020512000e5
:107150006134220080087800e04f20008134220052
:1071600080087800b04e2000a1342200800878000a
:10717000304c2000c134220080087800304b2000c1
:10718000e1342200800878002049200001352200e7
:1071900080087800c0472000213522008008780050
:1071a00060472000413522008008780020462000fa
:1071b00061352200800878002045200081352200ba
:1071c00080087800d0432000a13522008008780094
:1071d000b0422000c1352200800878009041200094
:1071e000e1352200800878000040200001362200ae
:1071f00080087800503c200021362200800878006a
:10720000603920004136220080087800e0352000f7
:10721000613622008008780060322000813622002a
:107220008008780020302000a136220080087800f5
:10723000702e2000c136220080087800302c2000fb
:10724000e136220080087800b02a200001372200b1
:1072500080087800702a20002137220080087800fa
:10726000902920004137220080087800c0292000a2
:107270006137220080087800a02920008137220091
:1072800080087800e02a2000a137220080087800da
:10729000c02c2000c137220080087800d02d2000ab
:1072a000e1372200800878005030200001382200a9
:1072b00080087800303220002138220080087800d1
:1072c000b03320004138220080087800503520007b
:1072d0006138220080087800e037200081382200e1
:1072e00080087800f03a2000a13822008008780059
:1072f000903f2000c13822008008780030442000f0
:10730000e13822008008780030472000013922004f
:1073100080087800204b2000213922008008780066
:10732000a04f20004139220080087800a05720009b
:107330006139220080087800006220008139220033
:1073400080087800c0682000a139220080087800f9
:1073500080732000c139220080087800507b200013
:10736000e139220080087800e07d2000013a220007
:1073700080087800e07b2000213a22008008780015
:10738000007c2000413a220080087800c07920006b
:10739000613a22008008780000762000813a2200bd
:1073a0008008780060772000a13a220080087800e9
:1073b00000732000c13a220080087800107020007d
:1073c000e13a220080087800206e2000013b220074
:1073d00080087800606b2000213b22008008780044
:1073e00060672000413b220080087800c0622000d6
:1073f000613b220080087800a05f2000813b2200d2
:1074000080087800e05b2000a13b22008008780023
:1074100050572000c13b220080087800604f2000b8
:10742000e13b220080087800f0482000013c220067
:1074300080087800f03b2000213c22008008780082
:10744000502f2000413c2200800878008029200035
:10745000613c220080087800e0242000813c22006a
:107460008008780090242000a13c22008008780049
:10747000d0222000c13c220080087800f0222000a9
:10748000e13c22008008780050212000013d2200cc
:1074900080087800e0222000213d2200800878004a
:1074a00080272000413d220080087800a02a20008b
:1074b000613d220080087800402e2000813d22009e
:1074c00080087800f02e2000a13d2200800878007e
:1074d000a02f2000c13d220080087800a02e2000af
:1074e000e13d220080087800902e2000013e22001d
:1074f00080087800402c2000213e2200800878007f
:1075000090282000413e220080087800302620008c
:10751000613e22008008780040222000813e220047
:107520008008780090212000a13e22008008780089
:1075300030202000c13e2200800878007021200009
:10754000e13e22008008780080212000013f2200d7
:107550008008780060232000213f22008008780006
:10756000b0242000413f22008008780080262000bf
:10757000613f220080087800c02a2000813f22005d
:107580008008780070302000a13f22008008780039
:10759000f0332000c13f22008008780070382000be
:1075a000e13f220080087800903b2000014022004b
:1075b00080087800603e200021402200800878008a
:1075c000b03f200041402200800878003041200078
:1075d0006140220080087800504020008140220055
:1075e00080087800c03e2000a1402200800878007a
:1075f000903e2000c140220080087800803d20009d
:10760000e140220080087800e03b20000141220098
:1076100080087800403a200021412200800878004c
:10762000303620004141220080087800b03120002f
:107630006141220080087800c02f20008141220093
:1076400080087800e02d2000a14122008008780009
:10765000202d2000c141220080087800e02c20006d
:10766000e141220080087800402b200001422200e6
:1076700080087800602b20002142220080087800da
:10768000502c20004142220080087800f02f20007a
:107690006142220080087800f031200081422200ff
:1076a00080087800f0352000a14222008008780090
:1076b00020392000c142220080087800f03d2000df
:1076c000e142220080087800e042200001432200cd
:1076d000800878003045200021432200800878008f
:1076e000f04920004143220080087800b04d20007e
:1076f000614322008008780020502000814322004e
:1077000080087800e0522000a14322008008780021
:1077100020542000c143220080087800f05320004c
:10772000e1432200800878004054200001442200f8
:1077300080087800805420002144220080087800ce
:10774000205320004144220080087800705120001e
:1077500061442200800878001050200081442200fb
:1077600080087800a04d2000a14422008008780005
:10777000104b2000c144220080087800804a20007d
:10778000e144220080087800f048200001452200f2
:1077900080087800204820002145220080087800d9
:1077a000e04620004145220080087800a0452000e6
:1077b0006145220080087800e044200081452200d5
:1077c00080087800a0432000a145220080087800ae
:1077d00020432000c145220080087800c0412000dd
:1077e000e145220080087800d03f200001462200b9
:1077f00080087800f03b20002146220080087800b5
:10780000e039200041462200800878000035200041
:107810006146220080087800f03220008146220074
:1078200080087800c02f2000a14622008008780040
:10783000d02d2000c146220080087800902c200026
:10784000e146220080087800702b200001472200ca
:1078500080087800b02b20002147220080087800a3
:10786000c02a20004147220080087800202a2000fa
:107870006147220080087800502a200081472200ba
:1078800080087800f02a2000a147220080087800b4
:10789000d02c2000c147220080087800102f200043
:1078a000e1472200800878002031200001482200b2
:1078b00080087800d032200021482200800878001b
:1078c000d033200041482200800878009035200005
:1078d0006148220080087800c038200081482200da
:1078e00080087800903a2000a148220080087800a3
:1078f000f03f2000c1482200800878000000060008
:1079000050402000e148220080087800f044200028
:107910000149220080087800704a20002149220095
:1079200080087800c051200041492200800878007a
:10793000805420006149220080087800b05c20005b
:10794000814922008008780020682000a149220097
:107950008008780060712000c1492200800878000a
:10796000d07e2000e149220080087800207e20009f
:10797000014a220080087800e07a2000214a220093
:107980008008780010742000414a220080087800a6
:10799000006d2000614a220080087800006320000a
:1079a000814a22008008780080642000a14a2200d9
:1079b00080087800c0652000c14a22008008780055
:1079c000f05e2000e14a2200800878001066200066
:1079d000014b22008008780050662000214b2200d5
:1079e0008008780060682000414b22008008780001
:1079f000e06c2000614b22008008780010742000a9
:107a0000814b22008008780000692000a14b2200f1
:107a100080087800106b2000c14b2200800878009d
:107a2000e06b2000e14b220080087800b06320006a
:107a3000014c220080087800505f2000214c220079
:107a400080087800b0522000414c22008008780065
:107a5000003e2000614c22008008780000302000a9
:107a6000814c220080087800e0262000a14c2200f2
:107a700080087800d0242000c14c220080087800c3
:107a8000f0232000e14c22008008780090242000a0
:107a9000014d220080087800c01a2000214d2200ec
:107aa0008008780020182000414d220080087800ce
:107ab000f0142000614d220080087800901a200008
:107ac000814d220080087800b0202000a14d2200c6
:107ad00080087800702c2000c14d220080087800ba
:107ae000a0292000e14d220080087800802220009b
:107af000014e220080087800801c2000214e2200c8
:107b000080087800201a2000414e2200800878006a
:107b100000112000614e2200800878003010200003
:107b2000814e220080087800a0152000a14e22007e
:107b30008008780000112000c14e220080087800e3
:107b400000112000e14e220080087800401d200036
:107b5000014f22008008780040222000214f22009f
:107b600080087800d0252000414f2200800878004e
:107b7000e02d2000614f220080087800a02e200018
:107b8000814f220080087800f0322000a14f2200af
:107b90008008780050412000c14f22008008780002
:107ba00020412000e14f220080087800c03e2000e4
:107bb00001502200800878009040200021502200cf
:107bc00080087800e04620004150220080087800bc
:107bd000004920006150220080087800304a2000cf
:107be0008150220080087800a0492000a150220086
:107bf0008008780010442000c150220080087800de
:107c0000c0402000e150220080087800403f200062
:107c10000151220080087800b0422000215122004a
:107c200080087800f041200041512200800878004f
:107c3000304220006151220080087800303c200052
:107c40008151220080087800a0382000a151220034
:107c500080087800302f2000c15122008008780071
:107c6000d0282000e15122008008780090202000d8
:107c70000152220080087800201a200021522200a0
:107c800080087800d011200041522200800878003e
:107c9000f01120006152220080087800a01220001c
:107ca000815222008008780000142000a152220096
:107cb00080087800c0162000c15222008008780099
:107cc00030192000e152220080087800501b20006b
:107cd00001532200800878008022200021532200d6
:107ce00080087800002a2000415322008008780094
:107cf000d03420006153220080087800503e2000dc
:107d0000815322008008780090492000a15322006e
:107d100080087800f04d2000c153220080087800d0
:107d2000304f2000e153220080087800104c2000e2
:107d30000154220080087800504e20002154220077
:107d400080087800304e20004154220080087800de
:107d50000058200061542200800878001054200050
:107d6000815422008008780070512000a154220024
:107d70008008780010512000c1542200800878004b
:107d800050572000e154220080087800c0542000a1
:107d900001552200800878008052200021552200e1
:107da00080087800c04f20004155220080087800ec
:107db000604920006155220080087800d04b2000e7
:107dc0008155220080087800e0512000a155220052
:107dd00080087800e0512000c1552200800878001a
:107de000704e2000e155220080087800504e20009f
:107df0000156220080087800004d20002156220004
:107e000080087800304e200041562200800878001b
:107e1000104f20006156220080087800b0452000f5
:107e2000815622008008780060472000a156220079
:107e300080087800a0452000c15622008008780004
:107e400030422000e15622008008780040442000a3
:107e50000157220080087800a03c20002157220012
:107e600080087800103820004157220080087800f0
:107e7000e03320006157220080087800e02f2000c6
:107e80008157220080087800f02d2000a1572200a1
:107e900080087800802d2000c157220080087800db
:107ea000402b2000e157220080087800c0292000e4
:107eb0000158220080087800102c20002158220050
:107ec0008008780020312000415822008008780086
:107ed000e02f200061582200800878001035200033
:107ee000815822008008780030392000a1582200f3
:107ef00080087800f03e2000c158220080087800f9
:107f0000e0412000e1582200800878006044200011
:107f10000159220080087800c04720002159220022
:107f200080087800605120004159220080087800c4
:107f3000e05420006159220080087800205f200072
:107f4000815922008008780060692000a159220030
:107f500080087800d0712000c15922008008780084
:107f6000307d2000e159220080087800e07c20006c
:107f7000015a220080087800b07b2000215a22009c
:107f800080087800e0732000415a220080087800c1
:107f9000806c2000615a22008008780080642000f4
:107fa000815a22008008780000662000a15a220031
:107fb0008008780030652000c15a220080087800cf
:107fc000d0632000e15a220080087800f06d200084
:107fd000015b220080087800c0672000215b22003e
:107fe00080087800a06b2000415b220080087800a8
:107ff000206f2000615b2200800878001073200051
:10800000815b220080087800406a2000a15b22008a
:1080100080087800206f2000c15b22008008780073
:10802000306c2000e15b2200800878006060200056
:10803000015c220080087800e05c2000215c2200c6
:1080400080087800e04a2000415c22008008780027
:10805000303b2000615c220080087800d02a20009c
:10806000815c220080087800d0252000a15c2200dd
:108070008008780020252000c15c2200800878005c
:1080800010232000e15c220080087800c02120003d
:10809000015d22008008780050192000215d220037
:1080a00080087800d0182000415d22008008780008
:1080b000f0142000615d220080087800b01d2000cf
:1080c000815d220080087800a0212000a15d2200af
:1080d00080087800002b2000c15d22008008780015
:1080e00070262000e15d220080087800b01f20008b
:1080f000015e220080087800b01b2000215e220073
:1081000080087800801a2000415e220080087800f4
:1081100050102000615e220080087800b01420001a
:10812000815e220080087800c0132000a15e22003a
:1081300080087800900f2000c15e2200800878003f
:1081400070112000e15e220080087800601e20008f
:10815000015f22008008780080232000215f220038
:108160008008780020272000415f220080087800e6
:1081700060302000615f220080087800e03120003c
:10818000815f22008008780000362000a15f220075
:1081900080087800403e2000c15f220080087800ff
:1081a000703b2000e15f220080087800f03a200058
:1081b00001602200800878006040200021602200d9
:1081c0008008780070472000416022008008780015
:1081d000204520006160220080087800704a20005d
:1081e0008160220080087800004a2000a1602200ff
:1081f0008008780020452000c160220080087800b7
:1082000020422000e160220080087800f043200036
:108210000161220080087800f045200021612200e1
:1082200080087800a0432000416122008008780087
:10823000104120006161220080087800a03c2000ed
:10824000816122008008780020362000a161220090
:108250008008780070292000c16122008008780021
:10826000b0232000e161220080087800401a20003d
:10827000016222008008780080162000216222001e
:108280008008780070102000416222008008780089
:10829000a013200061622200800878007012200084
:1082a000816222008008780020152000a16222004f
:1082b00080087800f0162000c16222008008780053
:1082c000801a2000e162220080087800501d200002
:1082d0000163220080087800c0262000216322006c
:1082e00080087800502e200041632200800878002a
:1082f000003a20006163220080087800f0402000ee
:108300008163220080087800904d2000a163220044
:1083100080087800f04f2000c163220080087800b8
:10832000d04e2000e163220080087800404b2000fe
:108330000164220080087800604f20002164220040
:1083400080087800305020004164220080087800c6
:10835000605720006164220080087800f0512000fe
:10836000816422008008780090512000a1642200de
:108370008008780040542000c16422008008780002
:10838000a0592000e164220080087800c05220003b
:108390000165220080087800b04e2000216522008f
:1083a00080087800804c2000416522008008780019
:1083b000e04b20006165220080087800504e2000cc
:1083c0008165220080087800b0522000a16522005b
:1083d00080087800c04f2000c16522008008780026
:1083e000704a2000e165220080087800704c20006f
:1083f0000166220080087800304d200021662200ae
:1084000080087800b0502000416622008008780083
:10841000f04c20006166220080087800b042200005
:10842000816622008008780000422000a1662200b8
:1084300080087800e03f2000c166220080087800b4
:1084400090402000e166220080087800d0402000a3
:108450000167220080087800003a2000216722008e
:1084600080087800b038200041672200800878003a
:10847000c03a20006167220080087800e0372000c1
:10848000816722008008780000302000a167220068
:108490008008780060312000c167220080087800e1
:1084a000a0302000e167220080087800a02a200088
:1084b0000168220080087800f02d20002168220049
:1084c00080087800c03020004168220080087800d1
:1084d000202f2000616822008008780050302000a2
:1084e000816822008008780090382000a16822006e
:1084f0008008780090402000c16822008008780041
:10850000d0402000e168220080087800a0452000cb
:108510000169220080087800e04a200021692200d9
:10852000800878009051200041692200800878007e
:10853000d05220006169220080087800005f20008e
:108540008169220080087800b0672000a1692200bc
:1085500080087800a0732000c1692200800878009c
:10856000d07d2000e169220080087800f07f2000a3
:10857000016a220080087800b0772000216a22007a
:1085800080087800506d2000416a22008008780041
:10859000506a2000616a220080087800b0642000e0
:1085a000816a22008008780020692000a16a2200e8
:1085b00080087800e0672000c16a22008008780007
:1085c00000652000e16a220080087800706c2000bd
:1085d000016b22008008780020672000216b2200b8
:1085e00080087800f06c2000416b22008008780041
:1085f000c0772000616b2200800878003076200070
:10860000816b22008008780020712000a16b22007d
:108610008008780040722000c16b2200800878003a
:1086200080682000e16b22008008780070612000e3
:10863000016c22008008780020562000216c220066
:108640008008780070422000416c22008008780089
:10865000b0342000616c220080087800102c2000cb
:10866000816c220080087800a0272000a16c2200e5
:108670008008780060252000c16c22008008780006
:1086800030252000e16c2200800878007022200054
:10869000016d220080087800b0192000216d2200b1
:1086a00080087800201d2000416d2200800878009d
:1086b000001b2000616d220080087800c01e200091
:1086c000816d22008008780010202000a16d22001a
:1086d00080087800202e2000c16d220080087800dc
:1086e000e02a2000e16d220080087800f0222000be
:1086f000016e220080087800e01e2000216e22001a
:1087000080087800d0192000416e2200800878008f
:10871000c00e2000616e220080087800001020004a
:10872000816e220080087800c0112000a16e220016
:1087300080087800100c2000c16e220080087800ac
:10874000200d2000e16e220080087800501c2000df
:10875000016f220080087800401e2000216f220057
:108760008008780030232000416f220080087800c4
:10877000502a2000616f220080087800402c2000e1
:10878000816f220080087800e0322000a16f220073
:1087900080087800403c2000c16f220080087800eb
:1087a000e0442000e16f220080087800404420006f
:1087b00001702200800878006044200021702200af
:1087c00080087800004b200041702200800878006b
:1087d000b04d20006170220080087800c04f20005a
:1087e0008170220080087800f04c2000a1702200e7
:1087f0008008780000492000c170220080087800bd
:10880000e0422000e170220080087800e03e200075
:10881000017122008008780040432000217122006d
:1088200080087800f0422000417122008008780022
:10883000f04120006171220080087800303d200066
:108840008171220080087800f0362000a17122009a
:108850008008780090282000c171220080087800ec
:10886000a0222000e171220080087800b01c2000c6
:1088700001722200800878009014200021722200ea
:1088800080087800200d20004172220080087800c6
:1088900040122000617222008008780080142000bd
:1088a000817222008008780090162000a1722200b8
:1088b00080087800301b2000c172220080087800f8
:1088c000601f2000e172220080087800d020200084
:1088d0000173220080087800e02320002173220029
:1088e00080087800c02b20004173220080087800a7
:1088f000503820006173220080087800c03d2000bd
:108900008173220080087800e0482000a1732200d3
:1089100080087800f04e2000c173220080087800a3
:10892000304f2000e173220080087800704d200055
:108930000174220080087800f04d2000217422008c
:1089400080087800404c20004174220080087800a4
:10895000b054200061742200800878007054200018
:108960008174220080087800c0522000a174220087
:1089700080087800a0512000c1742200800878008f
:1089800080562000e174220080087800e051200029
:1089900001752200800878002051200021752200f6
:1089a00080087800905020004175220080087800ef
:1089b000e04d20006175220080087800104e2000f4
:1089c0008175220080087800f0502000a1752200f7
:1089d00080087800a04d2000c17522008008780032
:1089e000b04d2000e175220080087800204e200064
:1089f0000176220080087800404d20002176220078
:108a000080087800304c20004176220080087800f1
:108a1000a04b20006176220080087800d04320001f
:108a20008176220080087800a0442000a1762200f0
:108a30008008780090462000c176220080087800e7
:108a4000b0422000e176220080087800a04020009b
:108a50000177220080087800403e20002177220024
:108a600080087800703b2000417722008008780061
:108a70007037200061772200800878005031200094
:108a80008177220080087800302d2000a177220015
:108a90008008780080302000c177220080087800ac
:108aa000002f2000e177220080087800b02d200000
:108ab0000178220080087800902f20002178220081
:108ac00080087800b03220004178220080087800c9
:108ad000a030200061782200800878004033200018
:108ae0008178220080087800b03a2000a178220026
:108af00080087800d03e2000c178220080087800ed
:108b000060422000e1782200800878009047200031
:108b10000179220080087800a04b200021792200f2
:108b200080087800a04b200041792200800878005e
:108b3000d05220006179220080087800a05d2000da
:108b4000817922008008780040642000a179220009
:108b500080087800f0712000c17922008008780038
:108b6000507c2000e179220080087800d07b200032
:108b7000017a220080087800a0752000217a220066
:108b80008008780080742000417a220080087800f4
:108b9000106c2000617a220080087800c0612000fb
:108ba000817a22008008780090672000a17a220054
:108bb00080087800e0642000c17a220080087800f4
:108bc00010672000e17a220080087800106f2000f2
:108bd000017b220080087800a06c2000217b22000d
:108be00080087800306d2000417b220080087800ea
:108bf000b0742000617b220080087800607620003d
:108c0000817b220080087800b0722000a17b2200c6
:108c100080087800d0722000c17b22008008780094
:108c2000a06a2000e17b220080087800005f20001d
:108c3000017c220080087800f0502000217c220076
:108c400080087800f03d2000417c220080087800f8
:108c5000b0312000617c220080087800002a2000ca
:108c6000817c22008008780000262000a17c220060
:108c700080087800b0222000c17c220080087800a3
:108c800050232000e17c220080087800601f200033
:108c9000017d220080087800e0192000217d22005b
:108ca00080087800f01e2000417d220080087800b6
:108cb000e01f2000617d220080087800a0222000b3
:108cc000817d22008008780010272000a17d2200ed
:108cd0008008780010322000c17d220080087800d2
:108ce000602b2000e17d22008008780070262000a3
:108cf000017e220080087800c01e2000217e220014
:108d000080087800e0162000417e2200800878006c
:108d1000600f2000617e220080087800b0102000e3
:108d2000817e220080087800a0112000a17e220010
:108d30008008780040092000c17e22008008780069
:108d400030102000e17e220080087800801b200087
:108d5000017f220080087800001f2000217f220070
:108d60008008780060242000417f2200800878007d
:108d7000c0262000617f2200800878006028200043
:108d8000817f22008008780080352000a17f2200aa
:108d90008008780050412000c17f220080087800c0
:108da00000412000e17f220080087800f04120008f
:108db0000180220080087800804520002180220068
:108dc00080087800f04b2000418022008008780065
:108dd000b04d20006180220080087800104f2000f4
:108de000818022008008780000492000a1802200b4
:108df00080087800c0452000c180220080087800eb
:108e0000b0432000e1802200800878001044200058
:108e10000181220080087800204520002181220065
:108e2000800878007044200041812200800878008a
:108e3000a03f20006181220080087800003c2000d3
:108e4000818122008008780040352000a181220025
:108e500080087800f0282000c18122008008780076
:108e6000f0242000e181220080087800a01a200070
:108e700001822200800878007011200021822200e7
:108e800080087800700e200041822200800878005f
:108e900050132000618222008008780020132000f7
:108ea000818222008008780070152000a1822200b3
:108eb00080087800b01b2000c18222008008780062
:108ec000301c2000e182220080087800901d2000e4
:108ed00001832200800878001023200021832200d3
:108ee00080087800402e200041832200800878000e
:108ef00000392000618322008008780000422000b1
:108f00008183220080087800204c2000a183220069
:108f100080087800504d2000c1832200800878002e
:108f2000204e2000e183220080087800704b200052
:108f30000184220080087800904f200021842200c4
:108f400080087800a04f200041842200800878002b
:108f5000005820006184220080087800805320009f
:108f6000818422008008780070502000a1842200b3
:108f70008008780040512000c184220080087800d9
:108f800070542000e1842200800878007053200093
:108f900001852200800878000053200021852200ee
:108fa00080087800204c200041852200800878004d
:108fb000e04920006185220080087800e04f200011
:108fc0008185220080087800d0512000a1852200f0
:108fd00080087800e04e2000c185220080087800db
:108fe000d04e2000e185220080087800f04e20005d
:108ff0000186220080087800a04d200021862200f2
:1090000080087800405220004186220080087800c5
:10901000104c2000618622008008780080462000e5
:10902000818622008008780010472000a186220057
:1090300080087800f0452000c18622008008780072
:1090400040442000e186220080087800d0422000c1
:109050000187220080087800a03e2000218722009e
:1090600080087800b03b200041872200800878000b
:1090700020362000618722008008780040302000e0
:109080008187220080087800402e2000a1872200de
:1090900080087800a0302000c18722008008780076
:1090a000902f2000e187220080087800002e200009
:1090b0000188220080087800b03220002188220038
:1090c00080087800e0322000418822008008780083
:1090d000e0302000618822008008780000362000ff
:1090e000818822008008780050392000a188220061
:1090f00080087800f03f2000c188220080087800b6
:109100000000060060582000e188220080087800f6
:10911000005e20000189220080087800e0612000c4
:1091200021892200800878001062200041892200f5
:109130008008780090622000618922008008780011
:10914000906a200081892200800878003075200014
:10915000a189220080087800e0722000c1892200e5
:1091600080087800a0632000e18922008008780050
:10917000a05a2000018a220080087800606920003f
:10918000218a220080087800307a2000418a22005b
:109190008008780000702000618a22008008780032
:1091a000e05d2000818a220080087800703b20006a
:1091b000a18a22008008780050422000c18a220043
:1091c0008008780040542000e18a2200800878005e
:1091d000805b2000018b220080087800e04b20009b
:1091e000218b22008008780090372000418b2200dc
:1091f00080087800d0332000618b2200800878003e
:10920000f0462000818b2200800878006054200006
:10921000a18b22008008780000542000c18b22001e
:1092200080087800a04d2000e18b220080087800a3
:10923000d0442000018c220080087800e04e2000fd
:10924000218c22008008780020642000418c2200bc
:1092500080087800406c2000618c22008008780033
:10926000b0652000818c220080087800d05e20004c
:10927000a18c220080087800005e2000c18c2200b2
:109280008008780010612000e18c220080087800be
:1092900010662000018d220080087800c054200054
:1092a000218d22008008780070492000418d220025
:1092b00080087800004d2000618d22008008780031
:1092c000a0582000818d22008008780020572000bf
:1092d000a18d220080087800c0582000c18d220096
:1092e00080087800a0522000e18d220080087800dc
:1092f000604e2000018e220080087800005520007a
:10930000218e220080087800b05d2000418e22006e
:109310008008780040572000618e22008008780085
:1093200020512000818e220080087800204b2000f0
:10933000a18e220080087800904c2000c18e22006f
:109340008008780080502000e18e2200800878009c
:10935000a0532000018f220080087800204b2000bd
:10936000218f22008008780020472000418f2200b2
:109370008008780020462000618f22008008780055
:10938000a0442000818f2200800878001043200034
:10939000a18f220080087800c0492000c18f2200e0
:1093a00080087800e04f2000e18f220080087800dc
:1093b000c05020000190220080087800204a200040
:1093c0002190220080087800004f20004190220068
:1093d0008008780080512000619022008008780089
:1093e000105120008190220080087800a0512000b8
:1093f000a190220080087800004f2000c190220038
:1094000080087800004b2000e1902200800878005e
:10941000604d200001912200800878005054200007
:1094200021912200800878005054200041912200b0
:1094300080087800005220006191220080087800a6
:10944000f0512000819122008008780050562000c1
:10945000a191220080087800f0572000c1912200dd
:1094600080087800205c2000e191220080087800cc
:10947000e05a20000192220080087800e058200085
:109480002192220080087800b05a200041922200e8
:1094900080087800706020006192220080087800c7
:1094a000005f20008192220080087800c05d2000cb
:1094b000a192220080087800a05d2000c1922200c5
:1094c00080087800805f2000e19222008008780008
:1094d000d06120000193220080087800e060200025
:1094e0002193220080087800705e200041932200c2
:1094f00080087800f05b20006193220080087800eb
:10950000405d20008193220080087800605c20008c
:10951000a193220080087800a05a2000c193220065
:109520008008780040572000e193220080087800ee
:10953000f05320000194220080087800005220009f
:10954000219422008008780040532000419422009a
:109550008008780020532000619422008008780061
:10956000f05020008194220080087800304f2000c5
:10957000a194220080087800804f2000c19422002e
:109580008008780040522000e19422008008780092
:10959000105420000195220080087800805420009b
:1095a0002195220080087800005520004195220076
:1095b000800878000056200061952200800878001d
:1095c000005820008195220080087800f059200082
:1095d000a195220080087800805a2000c1952200c1
:1095e00080087800205b2000e19522008008780048
:1095f000105c20000196220080087800205d200089
:109600002196220080087800c05d2000419622004b
:1096100080087800205d2000619622008008780094
:10962000805b20008196220080087800e0592000ad
:10963000a196220080087800e0582000c196220000
:109640008008780020562000e196220080087800eb
:10965000505320000197220080087800f05020002d
:109660002197220080087800b04e20004197220008
:1096700080087800804c20006197220080087800e4
:10968000304a20008197220080087800204720007f
:10969000a197220080087800e0422000c1972200b4
:1096a00080087800303f2000e19722008008780091
:1096b000203e200001982200800878009041200080
:1096c0002198220080087800c0482000419822009c
:1096d00080087800a04e2000619822008008780061
:1096e000704e20008198220080087800404f2000b2
:1096f000a198220080087800a0552000c19822007f
:1097000080087800405b2000e19822008008780003
:10971000605f20000199220080087800f06020003e
:109720002199220080087800606020004199220081
:109730008008780000642000619922008008780089
:10974000106f200081992200800878003076200078
:10975000a199220080087800b06d2000c1992200f4
:1097600080087800405d2000e199220080087800a0
:1097700050592000019a2200800878006071200072
:10978000219a220080087800f07f2000419a220070
:1097900080087800506d2000619a220080087800cf
:1097a00060442000819a220080087800203d20003b
:1097b000a19a22008008780040502000c19a22001f
:1097c00080087800305c2000e19a22008008780050
:1097d000d04f2000019b22008008780080402000ac
:1097e000219b220080087800502e2000419b2200ff
:1097f00080087800b0362000619b22008008780045
:10980000904d2000819b2200800878002057200086
:10981000a19b22008008780040502000c19b2200bc
:1098200080087800704b2000e19b220080087800bf
:1098300020472000019c220080087800f05520007d
:10984000219c22008008780050682000419c220062
:1098500080087800906c2000619c220080087800cd
:10986000d05f2000819c220080087800905a200060
:10987000a19c220080087800505e2000c19c22003c
:109880008008780050642000e19c22008008780065
:10989000d0642000019d220080087800004d200047
:1098a000219d220080087800a0482000419d2200d0
:1098b0008008780040502000619d220080087800d8
:1098c000e05b2000819d2200800878000058200085
:1098d000a19d220080087800c0562000c19d220072
:1098e00080087800104c2000e19d2200800878005c
:1098f00050532000019e220080087800105b200059
:10990000219e220080087800c05c2000419e220039
:109910008008780010512000619e220080087800a5
:10992000804c2000819e220080087800604b20003f
:10993000a19e220080087800104e2000c19e2200c7
:109940008008780080522000e19e22008008780084
:10995000c0512000019f220080087800b0482000fc
:10996000219f22008008780080462000419f22002d
:109970008008780000472000619f2200800878005e
:1099800070442000819f220080087800a0442000bd
:10999000a19f220080087800604b2000c19f220018
:1099a0008008780060502000e19f22008008780045
:1099b000904f200001a0220080087800a04a2000db
:1099c00021a02200800878000051200041a0220040
:1099d00080087800b050200061a022008008780044
:1099e0009050200081a02200800878005051200073
:1099f000a1a0220080087800304e2000c1a02200e3
:109a000080087800c04a2000e1a022008008780089
:109a1000204f200001a1220080087800c0542000bf
:109a200021a12200800878002052200041a12200bc
:109a300080087800f051200061a1220080087800a1
:109a4000d053200081a122008008780020572000f8
:109a5000a1a122008008780070592000c1a1220035
:109a600080087800605c2000e1a122008008780076
:109a7000c058200001a222008008780090582000e1
:109a800021a2220080087800205c200041a2220050
:109a9000800878009060200061a222008008780091
:109aa000105e200081a2220080087800a05d2000c6
:109ab000a1a2220080087800805e2000c1a22200be
:109ac0008008780010602000e1a222008008780061
:109ad000f061200001a322008008780010602000bf
:109ae00021a3220080087800805d200041a322008d
:109af00080087800405c200061a322008008780084
:109b0000905d200081a3220080087800105c200076
:109b1000a1a3220080087800005a2000c1a32200df
:109b20008008780000572000e1a322008008780018
:109b3000b053200001a4220080087800c052200009
:109b400021a42200800878008053200041a4220034
:109b5000800878007052200061a4220080087800fc
:109b60006050200081a4220080087800f04e200080
:109b7000a1a422008008780010512000c1a4220076
:109b80008008780060532000e1a42200800878005b
:109b90000054200001a522008008780060542000b5
:109ba00021a52200800878006055200041a52200f0
:109bb000800878001057200061a5220080087800f6
:109bc0008058200081a5220080087800805920005c
:109bd000a1a5220080087800d0592000c1a522004c
:109be00080087800e05a2000e1a522008008780073
:109bf000605c200001a6220080087800905d2000b3
:109c000021a6220080087800c05d200041a6220025
:109c100080087800605d200061a62200800878003e
:109c2000c05b200081a6220080087800005a200036
:109c3000a1a6220080087800f0582000c1a62200ca
:109c40008008780020562000e1a6220080087800d5
:109c5000c052200001a72200800878003050200068
:109c600021a7220080087800004e200041a7220092
:109c700080087800c04b200061a72200800878008f
:109c8000004a200081a72200800878003047200089
:109c9000a1a722008008780090422000c1a72200de
:109ca00080087800503e2000e1a72200800878005c
:109cb000703e200001a8220080087800a044200007
:109cc00021a8220080087800c04c200041a8220072
:109cd00080087800b04f200061a82200800878003a
:109ce000d04d200081a8220080087800a0512000db
:109cf000a1a822008008780010562000c1a82200e8
:109d000080087800305c2000e1a8220080087800fc
:109d10004060200001a92200800878001061200026
:109d200021a92200800878004060200041a922007b
:109d300080087800b065200061a9220080087800c2
:109d40000072200081a9220080087800f0762000af
:109d5000a1a9220080087800406b2000c1a9220040
:109d600080087800705c2000e1a92200800878005b
:109d7000a05d200001aa220080087800d074200095
:109d800021aa220080087800107a200041aa22002f
:109d9000800878003065200061aa220080087800e1
:109da000103f200081aa220080087800603f200038
:109db000a1aa22008008780060512000c1aa2200d8
:109dc00080087800805c2000e1aa220080087800ea
:109dd000804c200001ab220080087800f03b20007e
:109de00021ab2200800878006030200041ab2200c7
:109df000800878002044200061ab220080087800b1
:109e0000e053200081ab22008008780070582000c9
:109e1000a1ab220080087800904e2000c1ab220048
:109e20008008780060452000e1ab220080087800bf
:109e3000204d200001ac220080087800605b2000eb
:109e400021ac220080087800306a200041ac22005a
:109e500080087800106b200061ac22008008780038
:109e6000805e200081ac22008008780080592000ac
:109e7000a1ac220080087800505e2000c1ac220016
:109e800080087800e0662000e1ac220080087800bd
:109e90005062200001ad220080087800a048200018
:109ea00021ad220080087800804a200041ad2200c8
:109eb000800878002052200061ad220080087800e0
:109ec000505c200081ad220080087800e05920001d
:109ed000a1ad220080087800a0532000c1ad22006f
:109ee00080087800d04a2000e1ad22008008780088
:109ef000c054200001ae220080087800405d2000a0
:109f000021ae2200800878008059200041ae220056
:109f1000800878003050200061ae22008008780070
:109f2000c04a200081ae220080087800604b2000eb
:109f3000a1ae22008008780040512000c1ae22006e
:109f400080087800a0542000e1ae2200800878004c
:109f5000104c200001af220080087800e04620006d
:109f600021af220080087800e046200041af2200a7
:109f7000800878002047200061af22008008780028
:109f80008044200081af2200800878003046200005
:109f9000a1af220080087800004b2000c1af220052
:109fa0008008780060502000e1af2200800878002f
:109fb000704f200001b0220080087800204b200064
:109fc00021b02200800878002051200041b02200fa
:109fd000800878008050200061b02200800878005e
:109fe0000051200081b0220080087800205120001c
:109ff000a1b0220080087800104e2000c1b02200dd
:10a0000080087800a04b2000e1b022008008780092
:10a010002050200001b122008008780080542000e8
:10a0200021b12200800878006052200041b1220056
:10a03000800878008052200061b1220080087800fa
:10a040000055200081b122008008780020572000b0
:10a05000a1b1220080087800205a2000c1b122005e
:10a0600080087800c05b2000e1b122008008780001
:10a070004059200001b2220080087800005a2000d8
:10a0800021b2220080087800a05e200041b22200a8
:10a0900080087800f05e200061b22200800878001d
:10a0a000305e200081b2220080087800e05d200050
:10a0b000a1b2220080087800105f2000c1b2220007
:10a0c00080087800b05f2000e1b2220080087800ac
:10a0d0007061200001b3220080087800805f2000ba
:10a0e00021b3220080087800c05d200041b3220027
:10a0f00080087800b05c200061b3220080087800fe
:10a10000505d200081b3220080087800a05b200011
:10a11000a1b322008008780040592000c1b322007a
:10a1200080087800c0562000e1b322008008780043
:10a130002053200001b4220080087800f052200053
:10a1400021b4220080087800c052200041b42200cf
:10a15000800878004052200061b422008008780016
:10a160000050200081b4220080087800504f200069
:10a17000a1b422008008780040512000c1b4220020
:10a180008008780040532000e1b422008008780065
:10a19000b053200001b5220080087800a0542000b0
:10a1a00021b5220080087800d055200041b522005a
:10a1b000800878002057200061b5220080087800d0
:10a1c0002059200081b522008008780080592000a5
:10a1d000a1b5220080087800805a2000c1b5220075
:10a1e00080087800e05b2000e1b52200800878005c
:10a1f000305d200001b6220080087800005e20005b
:10a2000021b6220080087800105e200041b62200ae
:10a2100080087800205d200061b622008008780068
:10a22000405b200081b6220080087800205a200080
:10a23000a1b6220080087800a0582000c1b62200f4
:10a240008008780030552000e1b6220080087800b0
:10a250001052200001b7220080087800e04f200053
:10a2600021b7220080087800904d200041b72200dd
:10a2700080087800704b200061b7220080087800c9
:10a280002049200081b7220080087800d0442000b7
:10a29000a1b722008008780010402000c1b722003a
:10a2a00080087800803d2000e1b722008008780017
:10a2b0009040200001b8220080087800204820004b
:10a2c00021b8220080087800a04e200041b822006a
:10a2d00080087800204e200061b8220080087800b5
:10a2e000904e200081b8220080087800d0542000d1
:10a2f000a1b8220080087800c05a2000c1b822000e
:10a3000080087800105f2000e1b822008008780003
:10a310006060200001b9220080087800f05f200012
:10a3200021b9220080087800f062200041b92200a3
:10a3300080087800e06d200061b922008008780074
:10a340008075200081b9220080087800d07120003b
:10a35000a1b9220080087800b0602000c1b92200b5
:10a360008008780080542000e1b92200800878003d
:10a370003062200001ba220080087800207d200091
:10a3800021ba220080087800707b200041ba2200a8
:10a3900080087800005c200061ba22008008780004
:10a3a0002040200081ba2200800878005049200017
:10a3b000a1ba220080087800a0552000c1ba22006e
:10a3c00080087800105a2000e1ba22008008780046
:10a3d0000049200001bb220080087800c03920001d
:10a3e00021bb220080087800b036200041bb22004b
:10a3f00080087800a04c200061bb22008008780013
:10a40000804e200081bb220080087800704c200024
:10a41000a1bb220080087800404b2000c1bb220075
:10a4200080087800f04d2000e1bb22008008780011
:10a43000404d200001bc2200800878008060200090
:10a4400021bc2200800878008062200041bc2200ec
:10a4500080087800a05e200061bc2200800878009f
:10a46000c05f200081bc2200800878004069200085
:10a47000a1bc22008008780080632000c1bc2200bb
:10a4800080087800305e2000e1bc2200800878005f
:10a49000905c200001bd220080087800005120005f
:10a4a00021bd220080087800404f200041bd2200dd
:10a4b00080087800e057200061bd22008008780005
:10a4c000e055200081bd2200800878003050200037
:10a4d000a1bd22008008780000552000c1bd2200e7
:10a4e0008008780070532000e1bd220080087800c9
:10a4f000f054200001be220080087800605820003f
:10a5000021be2200800878006056200041be220053
:10a51000800878001050200061be2200800878007a
:10a52000d04f200081be220080087800e05020003b
:10a53000a1be220080087800d04c2000c1be2200bd
:10a5400080087800b04f2000e1be2200800878002b
:10a55000f04d200001bf220080087800c04b200091
:10a5600021bf2200800878007049200041bf2200ee
:10a5700080087800d048200061bf22008008780061
:10a580006041200081bf220080087800a0412000a7
:10a59000a1bf220080087800904a2000c1bf22009d
:10a5a0008008780020532000e1bf22008008780056
:10a5b000b050200001c02200800878002048200010
:10a5c00021c0220080087800404e200041c02200b7
:10a5d00080087800204f200061c0220080087800a9
:10a5e0002052200081c02200800878000054200002
:10a5f000a1c022008008780040502000c1c0220085
:10a600008008780090492000e1c02200800878008e
:10a61000004c200001c12200800878004054200036
:10a6200021c1220080087800c055200041c12200cd
:10a6300080087800c052200061c1220080087800a4
:10a640002053200081c1220080087800605520003e
:10a65000a1c1220080087800a0572000c1c12200bb
:10a6600080087800c05d2000e1c1220080087800e9
:10a67000605c200001c2220080087800205a20007f
:10a6800021c2220080087800305b200041c22200f5
:10a6900080087800d05e200061c222008008780027
:10a6a0001060200081c22200800878003061200004
:10a6b000a1c2220080087800905f2000c1c2220061
:10a6c00080087800205e2000e1c222008008780027
:10a6d000705f200001c322008008780080602000a5
:10a6e00021c3220080087800405f200041c322007f
:10a6f00080087800005c200061c322008008780098
:10a70000f05a200081c3220080087800605a20009f
:10a71000a1c322008008780040592000c1c3220054
:10a720008008780040582000e1c3220080087800ab
:10a73000f054200001c4220080087800d05120008d
:10a7400021c42200800878008051200041c42200ea
:10a75000800878006052200061c4220080087800e0
:10a76000b051200081c42200800878008050200071
:10a77000a1c4220080087800b0502000c1c422008b
:10a780008008780080522000e1c422008008780010
:10a79000b053200001c52200800878002056200018
:10a7a00021c52200800878006057200041c52200a2
:10a7b000800878000057200061c5220080087800da
:10a7c0009057200081c5220080087800d0592000d1
:10a7d000a1c5220080087800a05c2000c1c522002d
:10a7e00080087800a05d2000e1c522008008780084
:10a7f000005d200001c6220080087800505c200027
:10a8000021c6220080087800205d200041c6220079
:10a8100080087800a05d200061c6220080087800d2
:10a82000d05b200081c622008008780040582000bc
:10a83000a1c622008008780010552000c1c6220061
:10a8400080087800e0522000e1c6220080087800ed
:10a850008051200001c7220080087800405020006d
:10a8600021c7220080087800a04d200041c72200a7
:10a8700080087800704a200061c7220080087800b4
:10a88000f048200081c7220080087800704720002f
:10a89000a1c722008008780080452000c1c722009f
:10a8a00080087800e0412000e1c72200800878009d
:10a8b000503f200001c8220080087800204220007c
:10a8c00021c8220080087800404a200041c82200a8
:10a8d00080087800b050200061c82200800878000d
:10a8e0002051200081c8220080087800e05120001b
:10a8f000a1c822008008780040552000c1c822006d
:10a900008008780000402000e1882200800878005c
:10a91000100020003090880031908000f01f20004f
:10a92000808f50001c003e000612ed0000067800eb
:10a930000c064600e088220060007e00a08f8800a0
:10a940003290800002014100e0882200600079001e
:10a95000f411b400329080004111dd00e188220042
:10a96000010141000009780032908000020141009d
:10a97000e0882200600079004100de003290800013
:10a980004111dd00e1882200010141000009780049
:10a990000632ec00e0ff390000000600e05620001f
:10a9a000e1c8220080087800c059200001c92200b7
:10a9b000800878004057200021c9220080087800d4
:10a9c000405b200041c922008008780060652000bb
:10a9d00061c92200800878002068200081c9220017
:10a9e0008008780090652000a1c9220080087800c6
:10a9f00080672000c1c9220080087800506b2000c9
:10aa0000e1c9220080087800306f200001ca2200ce
:10aa1000800878002075200021ca22008008780074
:10aa2000a07a200041ca220080087800907d200092
:10aa300061ca220080087800307a200081ca220092
:10aa400080087800206f2000a1ca220080087800ca
:10aa5000a0662000c1ca220080087800306620006d
:10aa6000e1ca220080087800f068200001cb2200b3
:10aa700080087800905a200021cb220080087800be
:10aa80008052200041cb220080087800804f2000b7
:10aa900061cb220080087800804d200081cb22000d
:10aaa00080087800004e2000a1cb220080087800aa
:10aab000e04c2000c1cb220080087800004220003a
:10aac000e1cb220080087800b038200001cc2200c1
:10aad00080087800a038200021cc2200800878006f
:10aae000703f200041cc22008008780020492000df
:10aaf00061cc220080087800e04b200081cc22004d
:10ab00008008780020412000a1cc22008008780035
:10ab100040422000c1cc220080087800004e200076
:10ab2000e1cc2200800878006058200001cd22008e
:10ab300080087800205e200021cd22008008780067
:10ab40003061200041cd220080087800e0552000cf
:10ab500061cd220080087800804d200081cd220048
:10ab600080087800a0552000a1cd22008008780040
:10ab700050642000c1cd220080087800a05c200035
:10ab8000e1cd220080087800f05a200001ce22009a
:10ab900080087800105a200021ce2200800878001a
:10aba000c058200041ce220080087800205a2000a2
:10abb00061ce2200800878005060200081ce220003
:10abc00080087800c05f2000a1ce220080087800b5
:10abd000c0502000c1ce220080087800b052200072
:10abe000e1ce2200800878009059200001cf220099
:10abf000800878006059200021cf2200800878006a
:10ac00004054200041cf220080087800004f2000ef
:10ac100061cf2200800878002043200081cf2200ed
:10ac20008008780020472000a1cf2200800878000b
:10ac300080572000c1cf220080087800c05c20002f
:10ac4000e1cf2200800878002052200001d02200ad
:10ac500080087800604a200021d022008008780017
:10ac6000c04f200041d0220080087800a05620006c
:10ac700061d0220080087800e05a200081d02200b4
:10ac800080087800a0522000a1d02200800878001f
:10ac900080472000c1d02200800878002043200097
:10aca000e1d0220080087800c045200001d12200b8
:10acb00080087800c043200021d12200800878005d
:10acc000703c200041d1220080087800203f200005
:10acd00061d12200800878000047200081d1220045
:10ace00080087800204d2000a1d122008008780043
:10acf000304b2000c1d1220080087800e0512000b4
:10ad0000e1d12200800878003050200001d22200da
:10ad100080087800c051200021d2220080087800ed
:10ad2000e053200041d222008008780030572000f4
:10ad300061d2220080087800d054200081d2220005
:10ad400080087800e0552000a1d222008008780019
:10ad500080602000c1d22200800878008068200036
:10ad6000e1d22200800878007066200001d3220022
:10ad700080087800205d200021d322008008780020
:10ad80005059200041d3220080087800d061200073
:10ad900061d3220080087800506b200081d322000c
:10ada0008008780040692000a1d322008008780044
:10adb00050682000c1d3220080087800706c200009
:10adc000e1d3220080087800e06c200001d422004a
:10add00080087800b068200021d422008008780024
:10ade0007062200041d42200800878007063200047
:10adf00061d4220080087800405a200081d42200cb
:10ae000080087800005d2000a1d42200800878002e
:10ae1000e05a2000c1d422008008780000592000a8
:10ae2000e1d4220080087800c057200001d522001c
:10ae300080087800405a200021d522008008780040
:10ae4000f056200041d5220080087800805520006f
:10ae500061d52200800878008055200081d522002d
:10ae60008008780050502000a1d52200800878008a
:10ae7000c04c2000c1d5220080087800d04a2000b4
:10ae8000e1d52200800878005049200001d6220038
:10ae900080087800c044200021d622008008780075
:10aea0004043200041d6220080087800f03e200078
:10aeb00061d62200800878006038200081d6220008
:10aec00080087800d0352000a1d6220080087800c4
:10aed000f03c2000c1d622008008780030412000dc
:10aee000e1d6220080087800e03e200001d7220051
:10aef00080087800b03c200021d72200800878002c
:10af0000b04d200041d72200800878006051200019
:10af100061d7220080087800c04e200081d722002f
:10af200080087800e0522000a1d722008008780035
:10af3000c0532000c1d7220080087800e04f2000d5
:10af4000e1d72200800878002052200001d822009a
:10af500080087800d054200021d822008008780092
:10af6000204e200041d8220080087800204b20008d
:10af700061d82200800878006050200081d822002b
:10af80008008780000512000a1d8220080087800b5
:10af900090522000c1d8220080087800b0582000cc
:10afa000e1d82200800878007058200001d92200e2
:10afb00080087800a058200021d92200800878005d
:10afc000e060200041d9220080087800006720005e
:10afd00061d92200800878002066200081d92200f3
:10afe00080087800f0662000a1d92200800878004f
:10aff00060692000c1d9220080087800306c2000f0
:10b00000e1d9220080087800f06f200001da2200e8
:10b01000800878007075200021da2200800878000e
:10b02000607a200041da220080087800907e2000bb
:10b0300061da220080087800b07b200081da2200eb
:10b0400080087800106f2000a1da220080087800c4
:10b05000c0632000c1da220080087800706a2000f6
:10b06000e1da220080087800b065200001db2200d0
:10b0700080087800c057200021db2200800878007b
:10b080006051200041db220080087800004f200042
:10b0900061db220080087800004d200081db220067
:10b0a00080087800e04f2000a1db220080087800b3
:10b0b000a0472000c1db220080087800103b200060
:10b0c000e1db2200800878000035200001dc22004e
:10b0d00080087800903b200021dc22008008780066
:10b0e0001046200041dc220080087800104d20002e
:10b0f00061dc2200800878000047200081dc22000b
:10b1000080087800a03e2000a1dc220080087800a2
:10b1100030492000c1dc2200800878006055200002
:10b12000e1dc220080087800f05e200001dd2200d2
:10b1300080087800e05f200021dd22008008780090
:10b140006056200041dd2200800878002048200061
:10b1500061dd220080087800c04a200081dd2200e5
:10b1600080087800705c2000a1dd22008008780053
:10b17000d0632000c1dd22008008780060592000e3
:10b18000e1dd220080087800c059200001de2200a5
:10b19000800878000059200021de22008008780015
:10b1a000605a200041de22008008780030612000d3
:10b1b00061de220080087800e064200081de220049
:10b1c0008008780020522000a1de2200800878004c
:10b1d000d0502000c1de22008008780050582000a6
:10b1e000e1de220080087800c05a200001df220042
:10b1f00080087800a054200021df22008008780019
:10b200002050200041df22008008780030432000d9
:10b2100061df2200800878004045200081df2200a5
:10b220008008780010542000a1df220080087800f8
:10b23000005d2000c1df22008008780080552000da
:10b24000e1df220080087800e04c200001e02200cd
:10b2500080087800f04d200021e02200800878006e
:10b26000c056200041e0220080087800805c200069
:10b2700061e0220080087800a056200081e02200d2
:10b2800080087800804a2000a1e022008008780031
:10b2900090442000c1e0220080087800a0472000f0
:10b2a000e1e0220080087800a047200001e12200b0
:10b2b00080087800f03d200021e12200800878001d
:10b2c0007039200041e1220080087800d03c200045
:10b2d00061e12200800878001049200081e122000d
:10b2e00080087800004f2000a1e12200800878004b
:10b2f000504b2000c1e1220080087800e04f200080
:10b30000e1e1220080087800404e200001e22200a6
:10b3100080087800c052200021e2220080087800d6
:10b320000057200041e2220080087800c058200029
:10b3300061e22200800878008053200081e2220030
:10b3400080087800c0582000a1e222008008780020
:10b3500050642000c1e2220080087800e0692000eb
:10b36000e1e22200800878007062200001e3220000
:10b37000800878004059200021e3220080087800ee
:10b38000305a200041e322008008780050682000f5
:10b3900061e3220080087800806c200081e32200b5
:10b3a00080087800106b2000a1e32200800878005c
:10b3b00070692000c1e3220080087800906b2000b3
:10b3c000e1e3220080087800f068200001e4220018
:10b3d000800878004067200021e42200800878007f
:10b3e000c064200041e4220080087800c05c200096
:10b3f00061e4220080087800e058200081e4220007
:10b4000080087800605c2000a1e4220080087800b9
:10b41000e05b2000c1e42200800878006059200031
:10b42000e1e42200800878002059200001e5220094
:10b43000800878008058200021e5220080087800ec
:10b44000c055200041e522008008780060562000a9
:10b4500061e52200800878000057200081e5220085
:10b460008008780090502000a1e522008008780034
:10b47000204b2000c1e5220080087800e049200030
:10b48000e1e52200800878006047200001e6220004
:10b49000800878006046200021e6220080087800bd
:10b4a0006042200041e6220080087800303b200006
:10b4b00061e6220080087800b033200081e6220097
:10b4c0008008780040382000a1e62200800878003b
:10b4d00040402000c1e62200800878004041200062
:10b4e000e1e6220080087800e03c200001e722002d
:10b4f00080087800a045200021e72200800878001d
:10b50000a050200041e7220080087800e04e200093
:10b5100061e72200800878000053200081e72200c4
:10b520008008780000552000a1e7220080087800fc
:10b53000b0512000c1e72200800878004050200070
:10b54000e1e7220080087800a052200001e82200f4
:10b55000800878000052200021e82200800878004e
:10b56000904c200041e8220080087800504e2000d6
:10b5700061e82200800878000050200081e8220065
:10b5800080087800804f2000a1e822008008780021
:10b5900060562000c1e8220080087800f0592000a1
:10b5a000e1e82200800878005057200001e92200dd
:10b5b00080087800d059200021e922008008780016
:10b5c000d061200041e9220080087800d065200089
:10b5d00061e92200800878006066200081e922008d
:10b5e0008008780030682000a1e9220080087800f7
:10b5f000f0692000c1e9220080087800f06c20008a
:10b60000e1e9220080087800c071200001ea2200f0
:10b61000800878007077200021ea220080087800f6
:10b62000707d200041ea220080087800007f200021
:10b6300061ea2200800878003076200081ea22004a
:10b640008008780010682000a1ea220080087800b5
:10b65000d0652000c1ea220080087800b06b20008d
:10b66000e1ea220080087800005d200001eb220062
:10b67000800878008054200021eb220080087800a8
:10b68000004e200041eb220080087800404d200051
:10b6900061eb220080087800f04d200081eb220051
:10b6a00080087800904e2000a1eb220080087800ee
:10b6b000c0402000c1eb22008008780050362000f6
:10b6c000e1eb220080087800f037200001ec220036
:10b6d000800878005042200021ec22008008780089
:10b6e000e04a200041ec220080087800404b200016
:10b6f00061ec2200800878005040200081ec22009c
:10b700008008780010402000a1ec2200800878001a
:10b71000604a2000c1ec2200800878000057200019
:10b72000e1ec220080087800b05e200001ed2200ec
:10b7300080087800805e200021ed220080087800db
:10b74000f052200041ed220080087800604920007e
:10b7500061ed2200800878001052200081ed220067
:10b7600080087800a0632000a1ed22008008780006
:10b77000805d2000c1ed22008008780090592000f3
:10b78000e1ed220080087800005a200001ee22003e
:10b7900080087800905a200021ee2200800878006e
:10b7a000a05c200041ee2200800878004064200068
:10b7b00061ee220080087800105c200081ee2200fb
:10b7c00080087800b04e2000a1ee220080087800aa
:10b7d00040542000c1ee220080087800005920006b
:10b7e000e1ee2200800878006056200001ef220080
:10b7f000800878003050200021ef22008008780077
:10b800000047200041ef22008008780020422000fd
:10b8100061ef220080087800804f200081ef220035
:10b8200080087800f05f2000a1ef220080087800f7
:10b83000905b2000c1ef220080087800e04d2000de
:10b84000e1ef220080087800204f200001f0220064
:10b85000800878009055200021f0220080087800b0
:10b86000e05b200041f0220080087800405c20006e
:10b8700061f0220080087800a052200081f02200b0
:10b880008008780030462000a1f02200800878006f
:10b8900020452000c1f0220080087800e04a200006
:10b8a000e1f02200800878002046200001f122000b
:10b8b000800878009039200021f12200800878006b
:10b8c000403a200041f122008008780080442000a6
:10b8d00061f1220080087800404f200081f12200b1
:10b8e00080087800d04d2000a1f122008008780067
:10b8f000604e2000c1f1220080087800a04d200099
:10b90000e1f1220080087800f04f200001f22200cf
:10b91000800878002057200021f22200800878005b
:10b920009059200041f22200800878000055200044
:10b9300061f2220080087800f055200081f2220098
:10b9400080087800d0602000a1f2220080087800f2
:10b9500070682000c1f2220080087800d0622000c8
:10b96000e1f2220080087800d058200001f3220084
:10b9700080087800e057200021f32200800878003a
:10b980009063200041f3220080087800f0682000d6
:10b9900061f3220080087800f069200081f3220022
:10b9a0008008780050692000a1f322008008780008
:10b9b000d06b2000c1f3220080087800306c20009a
:10b9c000e1f3220080087800f068200001f42200f2
:10b9d00080087800b063200021f4220080087800fd
:10b9e0003063200041f4220080087800605b200072
:10b9f00061f4220080087800c05b200081f42200fe
:10ba000080087800005c2000a1f422008008780003
:10ba1000505a2000c1f4220080087800f05720001e
:10ba2000e1f4220080087800205a200001f522006d
:10ba3000800878004058200021f522008008780016
:10ba40000056200041f52200800878009056200022
:10ba500061f52200800878006052200081f5220004
:10ba600080087800204e2000a1f522008008780090
:10ba7000604b2000c1f5220080087800704920004a
:10ba8000e1f5220080087800a045200001f62200a0
:10ba9000800878000044200021f622008008780009
:10baa000a040200041f62200800878007038200075
:10bab00061f62200800878006034200081f62200c0
:10bac0008008780060392000a1f622008008780004
:10bad00060402000c1f6220080087800a0422000cb
:10bae000e1f6220080087800c041200001f7220022
:10baf00080087800304c200021f722008008780070
:10bb0000604e200041f7220080087800005020009d
:10bb100061f72200800878000057200081f722009a
:10bb20008008780010552000a1f7220080087800d6
:10bb300020512000c1f7220080087800e04e20004c
:10bb4000e1f7220080087800e051200001f822008f
:10bb5000800878005050200021f8220080087800ea
:10bb6000104e200041f8220080087800a04e2000ee
:10bb700061f8220080087800804e200081f82200c1
:10bb800080087800804f2000a1f82200800878000b
:10bb900090572000c1f8220080087800605a2000e9
:10bba000e1f8220080087800c058200001f9220046
:10bbb00080087800105d200021f9220080087800bc
:10bbc0003062200041f9220080087800a065200042
:10bbd00061f9220080087800f067200081f92200d6
:10bbe00080087800706a2000a1f92200800878009f
:10bbf000b06a2000c1f9220080087800106e200091
:10bc0000e1f92200800878008073200001fa220008
:10bc100080087800007b200021fa2200800878004c
:10bc2000f07f200041fa220080087800b07b2000dd
:10bc300061fa220080087800206e200081fa22003c
:10bc400080087800b0632000a1fa22008008780004
:10bc5000f06b2000c1fa22008008780060662000a6
:10bc6000e1fa220080087800a058200001fb2200a1
:10bc7000800878003050200021fb220080087800e6
:10bc8000704e200041fb220080087800604d2000ab
:10bc900061fb2200800878004051200081fb2200d7
:10bca00080087800304d2000a1fb22008008780039
:10bcb000403f2000c1fb2200800878003035200082
:10bcc000e1fb2200800878005039200001fc2200ae
:10bcd000800878007044200021fc22008008780051
:10bce000f04c200041fc220080087800c049200070
:10bcf00061fc220080087800903d200081fc220039
:10bd00008008780020442000a1fc220080087800f0
:10bd100000502000c1fc220080087800e05b200079
:10bd2000e1fc220080087800905e200001fd2200e6
:10bd300080087800005c200021fd22008008780047
:10bd4000404d200041fd220080087800904d2000e9
:10bd500061fd220080087800605b200081fd2200e8
:10bd60008008780040652000a1fd2200800878004e
:10bd7000505a2000c1fd220080087800c05a2000df
:10bd8000e1fd220080087800f057200001fe22002b
:10bd9000800878004059200021fe220080087800a9
:10bda000f05d200041fe2200800878002064200021
:10bdb00061fe2200800878007050200081fe220081
:10bdc00080087800b04e2000a1fe22008008780094
:10bdd00000552000c1fe2200800878008058200015
:10bde000e1fe2200800878002050200001ff2200a0
:10bdf00080087800004a200021ff22008008780097
:10be00008040200041ff220080087800c0452000cb
:10be100061ff220080087800d058200081ff2200b6
:10be200080087800b0632000a1ff2200800878001d
:10be300020552000c1ff220080087800204c2000ff
:10be4000e1ff220080087800105320000100230049
:10be50008008780010582000210023008008780016
:10be6000105d20004100230080087800405720002a
:10be70006100230080087800c04820008100230072
:10be80008008780020432000a1002300800878006b
:10be9000204d2000c100230080087800604c200065
:10bea000e100230080087800103e200001012300fb
:10beb00080087800003720002101230080087800e6
:10bec000903e20004101230080087800004c2000b3
:10bed0006101230080087800e053200081012300e5
:10bee00080087800f04c2000a10123008008780031
:10bef000304c2000c101230080087800004c200055
:10bf0000e101230080087800205620000102230070
:10bf100080087800605a2000210223008008780001
:10bf200040582000410223008008780090522000f1
:10bf30006102230080087800805a200081022300db
:10bf40008008780090662000a10223008008780015
:10bf5000c0672000c102230080087800105b200029
:10bf6000e1022300800878008054200001032300b0
:10bf700080087800005a2000210323008008780000
:10bf8000506420004103230080087800606720008f
:10bf9000610323008008780050672000810323009c
:10bfa0008008780050672000a103230080087800f3
:10bfb000506c2000c10323008008780080712000ad
:10bfc000e103230080087800306920000104230089
:10bfd00080087800e05e20002104230080087800bb
:10bfe000f06120004104230080087800c05d20003b
:10bff0006104230080087800805d20008104230014
:10c0000080087800005a2000a104230080087800ee
:10c0100090572000c104230080087800c0552000fc
:10c02000e104230080087800605c20000105230003
:10c0300080087800c058200021052300800878007f
:10c04000605420004105230080087800d052200071
:10c05000610523008008780020502000810523001e
:10c0600080087800f04c2000a105230080087800ab
:10c07000a04c2000c105230080087800c0482000a3
:10c08000e1052300800878006042200001062300bb
:10c0900080087800404220002106230080087800b4
:10c0a00020412000410623008008780080392000cc
:10c0b0006106230080087800c03720008106230035
:10c0c00080087800503f2000a106230080087800f7
:10c0d00010442000c1062300800878004041200061
:10c0e000e106230080087800303b20000107230090
:10c0f000800878006047200021072300800878002e
:10c100006051200041072300800878002051200062
:10c110006107230080087800604f2000810723001a
:10c1200080087800f0542000a107230080087800e0
:10c13000404e2000c10723008008780040502000b6
:10c14000e107230080087800a054200001082300a4
:10c1500080087800705320002108230080087800b0
:10c16000804a20004108230080087800a04d20006c
:10c170006108230080087800a05220008108230075
:10c1800080087800a0532000a108230080087800d0
:10c1900040552000c108230080087800f03f2000af
:10c1a000e1c822008008780010002000309088004c
:10c1b00031908000f01f2000808f50001c003e0056
:10c1c0000612ed00000678000c064600e0c82200ca
:10c1d00060007e00a08f8800329080000201410044
:10c1e000e0c8220060007900f411b40032908000b1
:10c1f0004111dd00e1c82200010141000009780081
:10c200003290800002014100e0c822006000790005
:10c210004100de00329080004111dd00e1c82200c3
:10c2200001014100000978000632ec00e0ff39000e
:10c23000000006008672ef00f0c1b3008652e300f2
:10c2400012003e00b2fd200093e4230086d2bf001e
:10c25000b1d2070037d20700bad007000001be00f4
:10c26000000020000120240032d207008bd20700fa
:10c2700061282100914078008180fb00e298230032
:10c28000807079008672ec00ebff39000000060038
:10c2900060ff2d00e11823008008780040362d0053
:10c2a000011923008008780070782c0021192300e0
:10c2b0008008780040c52b004119230080087800d1
:10c2c000201c2b006119230080087800807c2a0044
:10c2d0008119230080087800d0e52900a1192300e6
:10c2e00080087800a0572900c11923008008780031
:10c2f00060d12800e119230080087800b05228009e
:10c30000011a23008008780020db2700211a23006f
:10c3100080087800406a2700411a230080087800ce
:10c32000b0ff2600611a230080087800209b2600b9
:10c33000811a230080087800303c2600a11a2300cf
:10c3400080087800a0e22500c11a23008008780048
:10c35000108e2500e11a230080087800403e250059
:10c36000011b230080087800f0f22400211b230029
:10c3700080087800d0ab2400411b2300800878009f
:10c38000b0682400611b2300800878005029240035
:10c39000811b23008008780090ed2300a11b23005f
:10c3a0008008780020b52300c11b23008008780096
:10c3b000d07f2300e11b230080087800904d2300ec
:10c3c000011c230080087800201e2300211c23006c
:10c3d0008008780050f12200411c2300800878007a
:10c3e00000c72200611c230080087800209f2200e3
:10c3f000811c23008008780070792200a11c230092
:10c4000080087800e0552200c11c230080087800d5
:10c4100060342200e11c230080087800b014220060
:10c42000011d230080087800c0f62100211d230093
:10c430008008780090da2100411d230080087800f0
:10c44000f0bf2100611d230080087800c0a62100f4
:10c45000811d230080087800108f2100a11d23007a
:10c4600080087800a0782100c11d23008008780092
:10c4700080632100e11d230080087800904f210097
:10c48000011e230080087800c03c2100211e2300eb
:10c4900080087800f02a2100411e230080087800df
:10c4a000301a2100611e230080087800500a210004
:10c4b000811e23008008780060fb2000a11e23005d
:10c4c0008008780040ed2000c11e2300800878001d
:10c4d000f0df2000e11e23008008780060d32000f8
:10c4e000011f23008008780080c72000211f23003f
:10c4f0008008780050bc2000411f2300800878008d
:10c50000c0b12000611f230080087800c0a7200070
:10c51000811f230080087800609e2000a11f230057
:10c520008008780080952000c11f230080087800d3
:10c53000108d2000e11f2300800878003085200046
:10c540000120230080087800b07d200021202300f6
:10c5500080087800a0762000412023008008780021
:10c56000007020006120230080087800b06920005e
:10c570008120230080087800c0632000a1202300d0
:10c5800080087800305e2000c120230080087800f9
:10c59000e0582000e120230080087800e0532000cc
:10c5a0000121230080087800304f20002121230042
:10c5b00080087800c04a20004121230080087800cc
:10c5c00090462000612123008008780090422000de
:10c5d0008121230080087800e03e2000a121230073
:10c5e00080087800503b2000c1212300800878009b
:10c5f00000382000e121230080087800e03420008a
:10c600000122230080087800e0312000212223004d
:10c6100080087800102f2000412223008008780035
:10c62000702c20006122230080087800f02920006f
:10c63000812223008008780090272000a122230077
:10c640008008780060252000c1222300800878003f
:10c6500040232000e12223008008780050212000a0
:10c660000123230080087800701f2000212323006d
:10c6700080087800b01d2000412323008008780046
:10c68000001c20006123230080087800701a20001d
:10c690008123230080087800f0182000a1232300c4
:10c6a0008008780090172000c123230080087800bc
:10c6b00040162000e12323008008780000152000a8
:10c6c0000124230080087800d013200021242300b7
:10c6d00080087800b01220004124230080087800f0
:10c6e000a01120006124230080087800a010200001
:10c6f0008124230080087800b00f2000a1242300ab
:10c7000080087800d00e2000c12423008008780023
:10c71000000e2000e124230080087800300d200066
:10c720000125230080087800800c200021252300ab
:10c7300080087800c00b2000412523008008780085
:10c74000200b20006125230080087800800a20004b
:10c750008125230080087800e0092000a12523001e
:10c760008008780050092000c12523008008780047
:10c77000d0082000e1252300800878005008200020
:10c780000126230080087800e007200021262300ee
:10c790008008780070072000412623008008780078
:10c7a000000720006126230080087800a0062000f2
:10c7b000812623008008780040062000a12623005f
:10c7c00080087800e0052000c1262300800878005a
:10c7d00090052000e1262300800878004005200015
:10c7e0000127230080087800f0042000212723007f
:10c7f00080087800b00420004127230080087800da
:10c800007004200061272300800878003004200095
:10c810008127230080087800f0032000a12723004f
:10c8200080087800b0032000c1272300800878002a
:10c8300080032000e12723008008780050032000b7
:10c8400001282300800878002003200021282300ed
:10c8500080087800f002200041282300800878003a
:10c86000c00220006128230080087800a002200078
:10c87000812823008008780080022000a12823005e
:10c880008008780050022000c1282300800878002a
:10c89000c00f2e00e148230080087800b0452d002d
:10c8a000014923008008780000872c0021492300db
:10c8b0008008780000d32b004149230080087800cd
:10c8c00020292b006149230080087800c0882a00b5
:10c8d000814923008008780060f12900a1492300e4
:10c8e0008008780080622900c14923008008780010
:10c8f000b0db2800e149230080087800705c280044
:10c90000014a23008008780040e42700214a2300e0
:10c9100080087800e0722700414a230080087800f0
:10c92000e0072700614a230080087800e0a2260083
:10c93000814a23008008780080432600a14a230012
:10c940008008780080e92500c14a2300800878002b
:10c9500090942500e14a2300800878006044250077
:10c96000014b230080087800b0f82400214b2300fd
:10c970008008780040b12400414b230080087800f3
:10c98000d06d2400614b230080087800302e2400f5
:10c99000814b23008008780020f22300a14b230064
:10c9a0008008780070b92300c14b2300800878000c
:10c9b000f0832300e14b23008008780070512300ae
:10c9c000014c230080087800c0212300214c230063
:10c9d00080087800c0f42200414c230080087800d1
:10c9e00040ca2200614c23008008780030a2220057
:10c9f000814c230080087800607c2200a14c230039
:10ca000080087800a0582200c14c230080087800dc
:10ca1000f0362200e14c2300800878002017220025
:10ca2000014d23008008780010f92100214d2300da
:10ca300080087800c0dc2100414d23008008780088
:10ca4000f0c12100614d230080087800b0a82100ca
:10ca5000814d230080087800e0902100a14d230043
:10ca600080087800607a2100c14d2300800878009a
:10ca700020652100e14d230080087800105121003d
:10ca8000014e230080087800303e2100214e230013
:10ca900080087800502c2100414e23008008780047
:10caa000701b2100614e230080087800900b21004c
:10cab000814e23008008780090fc2000a14e2300c6
:10cac0008008780060ee2000c14e230080087800c6
:10cad00000e12000e14e23008008780060d42000af
:10cae000014f23008008780070c82000214f2300e8
:10caf0008008780030bd2000414f23008008780076
:10cb000090b22000614f23008008780090a8200098
:10cb1000814f230080087800109f2000a14f230040
:10cb20008008780030962000c14f230080087800ec
:10cb3000c08d2000e14f230080087800c0852000d0
:10cb40000150230080087800407e200021502300ff
:10cb5000800878003077200041502300800878005a
:10cb6000807020006150230080087800306a200027
:10cb7000815023008008780030642000a1502300f9
:10cb800080087800905e2000c15023008008780063
:10cb900050592000e15023008008780040542000c4
:10cba0000151230080087800904f2000215123007c
:10cbb00080087800104b2000415123008008780045
:10cbc000e04620006151230080087800e042200008
:10cbd0008151230080087800203f2000a1512300cc
:10cbe00080087800903b2000c15123008008780025
:10cbf00040382000e15123008008780010352000e3
:10cc000001522300800878002032200021522300a6
:10cc100080087800502f20004152230080087800bf
:10cc2000a02c20006152230080087800202a2000d8
:10cc30008152230080087800c0272000a1522300e1
:10cc40008008780090252000c152230080087800d9
:10cc500070232000e152230080087800702120001a
:10cc60000153230080087800901f200021532300e7
:10cc700080087800d01d20004153230080087800f0
:10cc8000201c20006153230080087800901a2000a7
:10cc9000815323008008780010192000a15323003d
:10cca00080087800a0172000c15323008008780076
:10ccb00050162000e1532300800878001015200052
:10ccc0000154230080087800e01320002154230041
:10ccd00080087800c01220004154230080087800aa
:10cce000b01120006154230080087800c01020009b
:10ccf0008154230080087800d00f2000a154230025
:10cd000080087800e00e2000c154230080087800dd
:10cd1000100e2000e154230080087800400d200010
:10cd20000155230080087800800c20002155230045
:10cd300080087800d00b200041552300800878003f
:10cd4000300b20006155230080087800900a2000f5
:10cd50008155230080087800f0092000a1552300a8
:10cd60008008780060092000c15523008008780001
:10cd7000e0082000e15523008008780060082000ca
:10cd80000156230080087800e00720002156230088
:10cd90008008780070072000415623008008780042
:10cda000000720006156230080087800a0062000bc
:10cdb000815623008008780040062000a1562300f9
:10cdc00080087800f0052000c15623008008780014
:10cdd00090052000e15623008008780040052000df
:10cde0000157230080087800000520002157230008
:10cdf00080087800b00420004157230080087800a4
:10ce0000700420006157230080087800300420005f
:10ce10008157230080087800f0032000a1572300e9
:10ce200080087800c0032000c157230080087800e4
:10ce300080032000e1572300800878005003200081
:10ce40000158230080087800200320002158230087
:10ce500080087800f0022000415823008008780004
:10ce6000d00220006158230080087800a002200032
:10ce7000815823008008780080022000a1582300f8
:10ce80008008780060022000c158230080087800e4
:10ce900090282e00e158230080087800205d2d00a6
:10cea0000159230080087800209d2c00215923007f
:10ceb00080087800e0e72b004159230080087800c3
:10cec000d03c2b006159230080087800609b2a0029
:10ced0008159230080087800f0022a00a15923001c
:10cee0008008780020732900c15923008008780049
:10cef00050eb2800e159230080087800306b2800af
:10cf0000015a23008008780030f22700215a2300bc
:10cf10008008780010802700415a2300800878009c
:10cf200040142700615a23008008780090ae260044
:10cf3000815a230080087800904e2600a15a2300d1
:10cf400080087800f0f32500c15a2300800878009b
:10cf5000609e2500e15a230080087800b04d25002e
:10cf6000015b23008008780080012500215b2300fd
:10cf70008008780090b92400415b23008008780085
:10cf8000b0752400615b2300800878009035240090
:10cf9000815b23008008780020f92300a15b230037
:10cfa0008008780000c02300c15b2300800878005f
:10cfb000208a2300e15b230080087800405723008b
:10cfc000015c23008008780040272300215c2300b7
:10cfd00080087800f0f92200415c23008008780086
:10cfe00030cf2200615c230080087800d0a62200a8
:10cff000815c230080087800c0802200a15c2300af
:10d0000080087800c05c2200c15c230080087800a2
:10d01000d03a2200e15c230080087800d01a220078
:10d02000015d23008008780090fc2100215d230031
:10d030008008780000e02100415d2300800878002e
:10d0400010c52100615d230080087800a0ab21009d
:10d05000815d230080087800a0932100a15d23005a
:10d0600080087800007d2100c15d230080087800e1
:10d07000a0672100e15d2300800878007053210043
:10d08000015e23008008780060402100215e2300bb
:10d0900080087800602e2100415e2300800878001f
:10d0a000701d2100615e230080087800600d210062
:10d0b000815e23008008780040fe2000a15e2300ee
:10d0c0008008780000f02000c15e2300800878000e
:10d0d00090e22000e15e230080087800d0d5200097
:10d0e000015f230080087800d0c92000215f230061
:10d0f0008008780080be2000415f2300800878000f
:10d10000d0b32000615f230080087800b0a9200020
:10d11000815f23008008780030a02000a15f2300f9
:10d120008008780030972000c15f230080087800d5
:10d13000b08e2000e15f230080087800b0862000d8
:10d140000160230080087800207f200021602300f8
:10d150008008780000782000416023008008780073
:10d16000407120006160230080087800f06a200090
:10d170008160230080087800f0642000a160230013
:10d1800080087800405f2000c1602300800878009c
:10d19000e0592000e160230080087800e05420007e
:10d1a00001612300800878001050200021612300d5
:10d1b00080087800a04b200041612300800878009f
:10d1c00060472000616123008008780060432000f0
:10d1d0008161230080087800903f2000a161230036
:10d1e00080087800003c2000c1612300800878009e
:10d1f000a0382000e161230080087800703520000d
:10d200000162230080087800703220002162230030
:10d2100080087800a02f2000416223008008780059
:10d22000f02c20006162230080087800702a200022
:10d23000816223008008780010282000a16223006a
:10d2400080087800d0252000c16223008008780083
:10d25000b0232000e162230080087800b021200084
:10d260000163230080087800d01f20002163230081
:10d2700080087800001e20004163230080087800a9
:10d28000501c20006163230080087800c01a200031
:10d29000816323008008780040192000a1632300e7
:10d2a00080087800d0172000c16323008008780030
:10d2b00080162000e16323008008780030152000ec
:10d2c00001642300800878000014200021642300fa
:10d2d00080087800e0122000416423008008780074
:10d2e000d01120006164230080087800d010200055
:10d2f0008164230080087800e00f2000a1642300ef
:10d3000080087800000f2000c164230080087800a6
:10d31000300e2000e164230080087800600d2000ba
:10d320000165230080087800a00c200021652300ff
:10d3300080087800e00b2000416523008008780019
:10d34000400b20006165230080087800a00a2000bf
:10d350008165230080087800000a2000a165230071
:10d360008008780070092000c165230080087800db
:10d37000f0082000e1652300800878007008200094
:10d380000166230080087800f00720002166230052
:10d39000800878008007200041662300800878001c
:10d3a000100720006166230080087800b006200086
:10d3b000816623008008780050062000a1662300c3
:10d3c00080087800f0052000c166230080087800fe
:10d3d000a0052000e16623008008780050052000a9
:10d3e00001672300800878000005200021672300e2
:10d3f00080087800c004200041672300800878007e
:10d400007004200061672300800878003004200049
:10d41000816723008008780000042000a1672300b2
:10d4200080087800c0032000c167230080087800ce
:10d4300090032000e167230080087800500320005b
:10d440000168230080087800200320002168230061
:10d4500080087800000320004168230080087800dd
:10d46000d00220006168230080087800a00220001c
:10d47000816823008008780080022000a1682300d2
:10d480008008780060022000c168230080087800ce
:10d4900020ef2d00e128230080087800f0262d00e1
:10d4a0000129230080087800006a2c00212923002c
:10d4b00080087800a0b72b0041292300800878005d
:10d4c000400f2b00612923008008780060702a003b
:10d4d000812923008008780060da2900a12923002f
:10d4e00080087800d04c2900c129230080087800ea
:10d4f00030c72800e129230080087800104928005f
:10d50000012a23008008780000d22700212a230066
:10d5100080087800a0612700412a23008008780055
:10d5200090f72600612a2300800878008093260067
:10d53000812a23008008780000352600a12a2300d4
:10d5400080087800d0db2500c12a230080087800fd
:10d55000a0872500e12a23008008780030382500c4
:10d56000012b23008008780030ed2400212b2300bc
:10d570008008780060a62400412b230080087800f2
:10d5800090632400612b230080087800802424000d
:10d59000812b23008008780000e92300a12b2300c1
:10d5a00080087800d0b02300c12b230080087800c9
:10d5b000d07b2300e12b230080087800c0492300a2
:10d5c000012c230080087800801a2300212c2300de
:10d5d00080087800e0ed2200412c230080087800cc
:10d5e000d0c32200612c230080087800109c220008
:10d5f000812c23008008780090762200a12c230043
:10d600008008780030532200c12c23008008780065
:10d61000d0312200e12c2300800878004012220043
:10d62000012d23008008780080f42100212d2300a3
:10d630008008780070d82100412d230080087800f0
:10d64000e0bd2100612d230080087800e0a42100c6
:10d65000812d230080087800408d2100a12d23001a
:10d6600080087800f0762100c12d23008008780022
:10d67000e0612100e12d230080087800104e210098
:10d68000012e230080087800503b2100212e23002a
:10d6900080087800a0292100412e2300800878000e
:10d6a000e0182100612e2300800878002009210065
:10d6b000812e23008008780040fa2000a12e23004c
:10d6c0008008780030ec2000c12e2300800878000c
:10d6d000f0de2000e12e23008008780070d22000c8
:10d6e000012f230080087800a0c62000212f2300ee
:10d6f0008008780080bb2000412f2300800878003c
:10d70000f0b02000612f23008008780000a72000df
:10d71000812f230080087800a09d2000a12f2300e6
:10d7200080087800d0942000c12f23008008780062
:10d73000708c2000e12f2300800878009084200066
:10d740000130230080087800207d20002130230054
:10d75000800878002076200041302300800878007f
:10d76000806f20006130230080087800306920003d
:10d77000813023008008780050632000a13023000e
:10d7800080087800c05d2000c13023008008780048
:10d7900080582000e130230080087800805320006a
:10d7a0000131230080087800d04e20002131230071
:10d7b00080087800604a200041312300800878000a
:10d7c000404620006131230080087800504220004c
:10d7d0008131230080087800903e2000a131230091
:10d7e00080087800103b2000c131230080087800b9
:10d7f000c0372000e131230080087800a0342000e9
:10d800000132230080087800a0312000213223005b
:10d8100080087800e02e2000413223008008780044
:10d82000402c20006132230080087800c0292000ad
:10d83000813223008008780070272000a132230065
:10d840008008780030252000c1322300800878004d
:10d8500020232000e13223008008780020212000ce
:10d860000133230080087800401f2000213323006b
:10d8700080087800801d2000413323008008780054
:10d88000e01b20006133230080087800501a20003c
:10d890008133230080087800d0182000a1332300b2
:10d8a0008008780070172000c133230080087800ba
:10d8b00020162000e133230080087800e0142000c7
:10d8c0000134230080087800b013200021342300a5
:10d8d00080087800a01220004134230080087800de
:10d8e00090112000613423008008780090102000ff
:10d8f0008134230080087800a00f2000a134230089
:10d9000080087800c00e2000c13423008008780011
:10d91000f00d2000e134230080087800200d200065
:10d920000135230080087800700c20002135230089
:10d9300080087800b00b2000413523008008780073
:10d94000100b20006135230080087800700a200049
:10d950008135230080087800e0092000a1352300ec
:10d960008008780050092000c13523008008780025
:10d97000c0082000e135230080087800500820000e
:10d980000136230080087800d007200021362300cc
:10d990008008780060072000413623008008780066
:10d9a000f0062000613623008008780090062000f1
:10d9b000813623008008780030062000a13623003d
:10d9c00080087800e0052000c13623008008780038
:10d9d00080052000e1362300800878004005200003
:10d9e0000137230080087800f0042000213723004d
:10d9f00080087800a00420004137230080087800c8
:10da00006004200061372300800878002004200093
:10da10008137230080087800f0032000a13723001d
:10da200080087800b0032000c13723008008780008
:10da300080032000e1372300800878005003200095
:10da400001382300800878002003200021382300bb
:10da500080087800f0022000413823008008780018
:10da6000c00220006138230080087800a002200056
:10da7000813823008008780070022000a13823003c
:10da80008008780050022000c13823008008780008
:10da900020d72d00e13823008008780040102d00a9
:10daa000013923008008780090542c00213923008c
:10dab0008008780060a32b0041392300800878009b
:10dac00030fc2a006139230080087800505e2a006b
:10dad000813923008008780060c92900a13923001a
:10dae00080087800c03c2900c139230080087800f4
:10daf00000b82800e139230080087800c03a2800e7
:10db0000013a23008008780080c42700213a2300ce
:10db100080087800e0542700413a2300800878000c
:10db200090eb2600613a23008008780020882600c8
:10db3000813a230080087800402a2600a13a230079
:10db400080087800b0d12500c13a23008008780011
:10db5000107e2500e13a230080087800302f250050
:10db6000013b230080087800b0e42400213b23001f
:10db700080087800609e2400413b230080087800e4
:10db8000005c2400613b230080087800601d2400b5
:10db9000813b23008008780040e22300a13b230062
:10dba0008008780070aa2300c13b23008008780019
:10dbb000c0752300e13b2300800878001044230057
:10dbc000013c23008008780020152300213c23001d
:10dbd00080087800e0e82200413c230080087800bb
:10dbe00010bf2200613c230080087800909722003b
:10dbf000813c23008008780050722200a13c230061
:10dc000080087800304f2200c13c23008008780053
:10dc1000002e2200e13c230080087800b00e220094
:10dc2000013d23008008780020f12100213d2300e0
:10dc30008008780040d52100413d2300800878000d
:10dc4000e0ba2100613d23008008780000a2210095
:10dc5000813d230080087800908a2100a13d2300a7
:10dc60008008780070742100c13d2300800878008e
:10dc7000805f2100e13d230080087800d04b210027
:10dc8000013e23008008780030392100213e230026
:10dc90008008780090272100413e2300800878000a
:10dca00000172100613e2300800878005007210002
:10dcb000813e23008008780090f82000a13e2300d8
:10dcc00080087800a0ea2000c13e23008008780088
:10dcd00070dd2000e13e23008008780000d12000a4
:10dce000013f23008008780050c52000213f230019
:10dcf0008008780030ba2000413f23008008780077
:10dd0000c0af2000613f230080087800e0a520001c
:10dd1000813f230080087800909c2000a13f2300d1
:10dd200080087800d0932000c13f2300800878004d
:10dd3000808b2000e13f230080087800b083200022
:10dd40000140230080087800407c2000214023000f
:10dd5000800878005075200041402300800878003a
:10dd6000c06e200061402300800878008068200099
:10dd70008140230080087800a0622000a140230099
:10dd800080087800205d2000c140230080087800d2
:10dd9000e0572000e140230080087800f052200086
:10dda0000141230080087800504e200021412300cb
:10ddb00080087800e0492000414123008008780075
:10ddc000c04520006141230080087800d041200038
:10ddd0008141230080087800203e2000a1412300db
:10dde00080087800a03a2000c14123008008780014
:10ddf00060372000e1412300800878004034200093
:10de00000142230080087800503120002142230085
:10de100080087800902e200041422300800878007e
:10de2000f02b200061422300800878008029200028
:10de3000814223008008780020272000a14223008f
:10de400080087800f0242000c14223008008780078
:10de5000e0222000e142230080087800f02020002a
:10de60000143230080087800101f20002143230075
:10de700080087800501d200041432300800878006e
:10de8000b01b20006143230080087800201a200086
:10de90008143230080087800b0182000a1432300ac
:10dea0008008780040172000c143230080087800d4
:10deb00000162000e143230080087800c0142000f1
:10dec000014423008008780090132000214423009f
:10ded00080087800801220004144230080087800e8
:10dee0007011200061442300800878007010200029
:10def0008144230080087800900f2000a144230073
:10df000080087800b00e2000c1442300800878000b
:10df1000d00d2000e144230080087800100d20007f
:10df20000145230080087800500c20002145230083
:10df300080087800a00b200041452300800878006d
:10df4000000b20006145230080087800600a200053
:10df50008145230080087800d0092000a1452300d6
:10df60008008780040092000c1452300800878001f
:10df7000c0082000e1452300800878004008200008
:10df80000146230080087800c007200021462300b6
:10df90008008780050072000414623008008780060
:10dfa000f0062000614623008008780090062000db
:10dfb000814623008008780030062000a146230017
:10dfc00080087800d0052000c14623008008780032
:10dfd00080052000e14623008008780030052000fd
:10dfe0000147230080087800e00420002147230037
:10dff00080087800a00420004147230080087800b2
:10e00000600420006147230080087800200420007d
:10e010008147230080087800e0032000a147230007
:10e0200080087800b0032000c147230080087800f2
:10e0300070032000e147230080087800400320009f
:10e0400001482300800878001003200021482300a5
:10e0500080087800f0022000414823008008780002
:10e06000c002200061482300800878009002200050
:10e07000814823008008780070022000a148230016
:10e080008008780050022000c148230080087800f2
:10e0900060992d00e168230080087800f0d52c00fd
:10e0a0000169230080087800901d2c00216923005d
:10e0b00080087800706f2b00416923008008780089
:10e0c00020cb2a00616923008008780010302a00e4
:10e0d0008169230080087800b09d2900a169230090
:10e0e0008008780080132900c16923008008780027
:10e0f00020912800e169230080087800001628009c
:10e10000016a230080087800e0a12700216a23002b
:10e110008008780030342700416a230080087800a6
:10e12000b0cc2600616a230080087800006b2600ce
:10e13000816a230080087800c00e2600a16a2300af
:10e1400080087800c0b72500c16a230080087800e5
:10e1500090652500e16a23008008780010182500ea
:10e16000016b230080087800e0ce2400216b23009f
:10e1700080087800c0892400416b23008008780063
:10e1800090482400616b230080087800000b240075
:10e19000816b230080087800f0d02300a16b23005e
:10e1a00080087800109a2300c16b23008008780053
:10e1b00050662300e16b230080087800803523003f
:10e1c000016c23008008780060072300216c230085
:10e1d00080087800e0db2200416c23008008780092
:10e1e000d0b22200616c230080087800008c2200ed
:10e1f000816c23008008780070672200a16c2300e6
:10e2000080087800e0442200c16c23008008780078
:10e2100040242200e16c2300800878008005220061
:10e22000016d23008008780070e82100216d230033
:10e230008008780010cd2100416d2300800878000f
:10e2400030b32100616d230080087800c09a21005e
:10e25000816d230080087800b0832100a16d230028
:10e2600080087800f06d2100c16d230080087800df
:10e2700060592100e16d23008008780000462100ec
:10e28000016e230080087800b0332100216e230046
:10e290008008780070222100416e230080087800f9
:10e2a00020122100616e230080087800c002210046
:10e2b000816e23008008780040f42000a16e2300c6
:10e2c0008008780080e62000c16e23008008780076
:10e2d00090d92000e16e23008008780060cd2000f6
:10e2e000016f230080087800e0c12000216f230027
:10e2f00080087800f0b62000416f23008008780085
:10e30000b0ac2000616f23008008780000a32000db
:10e31000816f230080087800e0992000a16f23001e
:10e320008008780040912000c16f230080087800a9
:10e3300010892000e16f23008008780060812000b0
:10e340000170230080087800207a200021702300cb
:10e350008008780040732000417023008008780016
:10e36000d06c20006170230080087800b066200027
:10e370008170230080087800f0602000a1702300e5
:10e3800080087800805b2000c1702300800878003e
:10e3900060562000e1702300800878008051200042
:10e3a0000171230080087800f04c200021712300c7
:10e3b00080087800a0482000417123008008780080
:10e3c000904420006171230080087800b040200054
:10e3d0008171230080087800103d2000a171230086
:10e3e00080087800a0392000c171230080087800df
:10e3f00060362000e171230080087800503320004f
:10e400000172230080087800703020002172230000
:10e4100080087800c02d2000417223008008780019
:10e42000302b20006172230080087800c028200073
:10e43000817223008008780070262000a1722300da
:10e440008008780050242000c172230080087800e2
:10e4500040222000e1722300800878006020200024
:10e460000173230080087800801e200021732300a0
:10e4700080087800d01c20004173230080087800b9
:10e48000301b20006173230080087800b019200041
:10e49000817323008008780040182000a1732300b6
:10e4a00080087800e0162000c173230080087800ff
:10e4b00090152000e173230080087800601420008c
:10e4c0000174230080087800401320002174230089
:10e4d0008008780020122000417423008008780012
:10e4e0002011200061742300800878003010200083
:10e4f0008174230080087800400f2000a17423005d
:10e5000080087800700e2000c17423008008780015
:10e51000a00d2000e174230080087800d00c2000ba
:10e520000175230080087800200c2000217523004d
:10e5300080087800700b2000417523008008780067
:10e54000d00a20006175230080087800300a20007e
:10e550008175230080087800a0092000a1752300a0
:10e560008008780010092000c17523008008780019
:10e5700090082000e1752300800878001008200032
:10e580000176230080087800a00720002176230070
:10e59000800878003007200041762300800878004a
:10e5a000d0062000617623008008780070062000e5
:10e5b000817623008008780010062000a1762300d1
:10e5c00080087800b0052000c1762300800878001c
:10e5d00060052000e17623008008780020052000f7
:10e5e0000177230080087800d004200021772300e1
:10e5f000800878009004200041772300800878008c
:10e600005004200061772300800878001004200067
:10e610008177230080087800d0032000a1772300b1
:10e6200080087800a0032000c177230080087800cc
:10e6300060032000e1772300800878003003200089
:10e64000017823008008780000032000217823004f
:10e6500080087800e00220004178230080087800dc
:10e66000b00220006178230080087800900220002a
:10e67000817823008008780060022000a1782300c0
:10e680008008780040022000c178230080087800cc
:10e6900060682e00e17823008008780060992d00e2
:10e6a0000179230080087800f0d52c00217923001f
:10e6b00080087800901d2c004179230080087800a4
:10e6c000706f2b00617923008008780020cb2a002e
:10e6d000817923008008780010302a00a179230076
:10e6e00080087800b09d2900c17923008008780057
:10e6f00080132900e1792300800878002091280008
:10e70000017a23008008780000162800217a23006f
:10e7100080087800e0a12700417a23008008780073
:10e7200030342700617a230080087800b0cc2600be
:10e73000817a230080087800006b2600a17a2300ec
:10e7400080087800c00e2600c17a23008008780077
:10e75000c0b72500e17a2300800878009065250085
:10e76000017b23008008780010182500217b2300fe
:10e7700080087800e0ce2400417b230080087800e8
:10e78000c0892400617b2300800878009048240021
:10e79000817b230080087800000b2400a17b2300ec
:10e7a00080087800f0d02300c17b23008008780027
:10e7b000109a2300e17b2300800878005066230034
:10e7c000017c23008008780080352300217c230011
:10e7d0008008780060072300417c230080087800cf
:10e7e000e0db2200617c230080087800d0b22200a8
:10e7f000817c230080087800008c2200a17c23000b
:10e800008008780070672200c17c230080087800af
:10e81000e0442200e17c23008008780040242200ac
:10e82000017d23008008780080052200217d2300df
:10e830008008780070e82100417d2300800878007e
:10e8400010cd2100617d23008008780030b32100c5
:10e85000817d230080087800c09a2100a17d2300db
:10e8600080087800b0832100c17d230080087800f3
:10e87000f06d2100e17d23008008780060592100bf
:10e88000017e23008008780000462100217e2300bd
:10e8900080087800b0332100417e23008008780092
:10e8a00070222100617e2300800878002012210060
:10e8b000817e230080087800c0022100a17e230011
:10e8c0008008780040f42000c17e23008008780092
:10e8d00080e62000e17e23008008780090d92000a7
:10e8e000017f23008008780060cd2000217f230075
:10e8f00080087800e0c12000417f23008008780074
:10e90000f0b62000617f230080087800b0ac2000c2
:10e91000817f23008008780000a32000a17f2300ce
:10e9200080087800e0992000c17f230080087800eb
:10e9300040912000e17f23008008780010892000aa
:10e94000018023008008780060812000218023005e
:10e9500080087800207a2000418023008008780019
:10e96000407320006180230080087800d06c200074
:10e970008180230080087800b0662000a1802300f9
:10e9800080087800f0602000c180230080087800b3
:10e99000805b2000e1802300800878006056200022
:10e9a000018123008008780080512000218123000c
:10e9b00080087800f04c2000418123008008780016
:10e9c000a048200061812300800878009044200046
:10e9d0008181230080087800b0402000a1812300bd
:10e9e00080087800103d2000c18123008008780055
:10e9f000a0392000e18123008008780060362000e3
:10ea000001822300800878005033200021822300f7
:10ea10008008780070302000418223008008780050
:10ea2000c02d20006182230080087800302b200058
:10ea30008182230080087800c0282000a182230062
:10ea40008008780070262000c182230080087800aa
:10ea500050242000e182230080087800402220001a
:10ea60000183230080087800602020002183230098
:10ea700080087800801e20004183230080087800f1
:10ea8000d01c20006183230080087800301b200008
:10ea90008183230080087800b0192000a18323001f
:10eaa0008008780040182000c18323008008780087
:10eab000e0162000e18323008008780090152000f4
:10eac0000184230080087800601420002184230042
:10ead00080087800401320004184230080087800db
:10eae000201220006184230080087800201120007b
:10eaf000818423008008780030102000a184230046
:10eb000080087800400f2000c1842300800878002e
:10eb1000700e2000e184230080087800a00d200002
:10eb20000185230080087800d00c20002185230077
:10eb300080087800200c20004185230080087800a0
:10eb4000700b20006185230080087800d00a200027
:10eb50008185230080087800300a2000a1852300e9
:10eb600080087800a0092000c18523008008780073
:10eb700010092000e185230080087800900820001b
:10eb800001862300800878001008200021862300d9
:10eb900080087800a00720004186230080087800c4
:10eba000300720006186230080087800d00620000e
:10ebb000818623008008780070062000a18623004b
:10ebc0008008780010062000c186230080087800a5
:10ebd000b0052000e1862300800878006005200051
:10ebe000018723008008780020052000218723006a
:10ebf00080087800d0042000418723008008780036
:10ec000090042000618723008008780050042000d1
:10ec1000818723008008780010042000a18723004a
:10ec200080087800d0032000c18723008008780086
:10ec3000a0032000e1872300800878006003200003
:10ec400001882300800878003003200021882300f9
:10ec500080087800000320004188230080087800a5
:10ec6000e00220006188230080087800b0022000c4
:10ec7000818823008008780090022000a18823006a
:10ec80008008780060022000c18823008008780096
:10ec900000000600e09a23000048eb0000c2b30029
:10eca000f19a230080487800f0c1b300019b230053
:10ecb00080487800e0c1b300119b230080487800b1
:10ecc000d0c1b300219b230080487800c0c1b300ad
:10ecd000319b230080487800b0c1b300419b2300e2
:10ece00080487800a0c1b300519b23008048780081
:10ecf00090c1b300619b23008048780080c1b300bd
:10ed0000719b23008048780070c1b300819b230071
:10ed10008048780060c1b300919b23008048780050
:10ed200050c1b300a19b23008048780040c1b300cc
:10ed3000b19b23008048780030c1b300c19b230001
:10ed40008048780020c1b300d19b23008048780020
:10ed500010c1b300e19b23008048780000c1b300dc
:10ed6000f19b230080487800f0c0b300019c230091
:10ed700080487800e0c0b300119c230080487800f0
:10ed8000d0c0b300219c230080487800c0c0b300ed
:10ed9000319c230080487800b0c0b300419c230020
:10eda00080487800a0c0b300519c230080487800c0
:10edb00090c0b300619c23008048780080c0b300fd
:10edc000719c23008048780070c0b300819c2300b0
:10edd0008048780060c0b300919c23008048780090
:10ede00050c0b300a19c23008048780040c0b3000d
:10edf000b19c23008048780030c0b300c19c230040
:10ee00008048780020c0b300d19c2300804878005f
:08ee100000000600ffff3700bf
:020000040000fa
:10ee1800f41100001000000080000000041200003f
:10ee28006400000080000000681200000c00000070
:10ee380080000000741200001a000000800000002a
:10ee48008e12000000260000800000008e380000ae
:0cee5800400100008000000000000000ed
:00000001FF
